:100000000C943C060C9464060C9464060C946406F0
:100010000C9464060C94FA260C9464060C94640602
:100020000C9464060C9464060C9464060C946406A8
:100030000C9464060C9464060C9464060C94640698
:100040000C9491250C9464060C9464060C9464063C
:100050000C9464060C9464060C9464060C94640678
:100060000C94DB250C94640600407A10F35A00A02F
:10007000724E18090010A5D4E80000E87648170071
:1000800000E40B54020000CA9A3B000000E1F505B1
:10009000000080969800000040420F000000A086FB
:1000A00001000000102700000000E803000000002D
:1000B0006400000000000A000000000001000000D1
:1000C00000002C76D888DC674F0823DFC1DFAE59EB
:1000D000E1B1B796E5E3E453C63AE651997696E87E
:1000E000E6C28426EB898C9B62ED407C6FFCEFBC02
:1000F0009C9F40F2BAA56FA5F490055A2AF75C932D
:100100006B6CF9676DC11BFCE0E40D47FEF520E662
:10011000B500D0ED902E0300943577050080841E45
:10012000080000204E0A000000C80C333333330FA0
:10013000986E12831141EF8D2114893BE65516CF3D
:10014000FEE6DB18D1844B381BF77C1D901DA4BB49
:10015000E424203284725E228100C9F124ECA1E5FE
:100160003D271200040304050406050D1B00FF16BD
:10017000FA160000000000016420060010F4002AB6
:1001800014AA14F6242825A1E260C4C8E460422B16
:100190004121002B0E9996FC33B6E6E081CDD81AAA
:1001A000002C0943F6CB116111012D0839F6FCF042
:1001B00081012E083316CC1151012F176A15F4B79F
:1001C000D9DCB2B965736364736373CBE696CDCD46
:1001D0000130156B15FC537573204173E5FF5737DC
:1001E000140732573500310D661BFCB384E2E06022
:1001F00066FF7F32196B15FC537573204173E5114F
:10020000DDC2B985737374EBE80E3E2833196BF5C4
:10021000FBF0833ABA75740BE90A2907F742EA84BE
:10022000E440C60600341B6B15FC33B8A1E042491C
:10023000C1852243223323332333071F540D6E031A
:10024000351D6B15FCF007811B1EC41C881C4CD08F
:100250005C590D2EB4B2BAA13890B9AA01361E6B02
:1002600015FC53757320417365B8F020E640E460D7
:1002700082E6CAAF6E280E64AE6A0037186B15FCB2
:10028000F00751464783EBE806D70D6E37B88E6E00
:10029000700A00381E6B15FC537573204173E5D549
:1002A0000DC581CC03099A89295FDD501CC85CD536
:1002B00000391F6B15FC537573204173E5573714D4
:1002C00007230732148383565637140732573500F5
:1002D0003A0BD376CC11510F18510100000004FFE6
:1002E000FF000000000000240027002A000000009A
:1002F00000250028002B0000000000230026002914
:1003000000040404040404040402020202020203BE
:1003100003030303030102040810204080010204C8
:10032000081020010204081020000000080002014B
:1003300000000304070000000000000000DC0003D0
:10034000020304040504060D00FE09FE0AFF016312
:1003500002CD040E200500DC0E210749858E4312D4
:1003600022079BB48EC412230E3D8C9E52920C4ADF
:1003700065504A4902240F4D84AE6C50A224DB9292
:100380002819B408250D4D849E48E998159316291F
:1003900001260E45849E2C8992AC124553A4042755
:1003A0000619B58E01280BDB7CAE244AA26E5116CD
:1003B000290CDB7C8E2CCAA22E5112012A0A2DA4F4
:1003C000AE4A65698A002B0A2D94AE301AA4300219
:1003D0002C079B7C1EA5042D060DA48E412E089B88
:1003E0007C9E6449002F0B4D84CE5A9815B330047F
:1003F000300C4D84AE2CA9794B6A1100310B4D8421
:10040000AE4C4AC29E0601320B4D849E25D3C2AC2F
:10041000E320330D4D848E41CC6A6BA8250B00344C
:100420000F4D84BE30939228292583162600350C63
:100430004D848E63C514865AB200360D4D849E25B8
:1004400013C321C96CC902370D4D848E41CCC22C17
:10045000CCC21A00380D4D849E25B3254B664B1631
:1004600000390D4D849E25B32543186AC9023A0B05
:10047000C37C9E64C9916449003B0AC37C9E64C9E5
:1004800011A5043C084D84CEAC6B073D0925948E24
:1004900041C706013E094D848EB45B47003F0D4DB8
:1004A000849E25D3C2AC98431100400D4D849E25F7
:1004B000332D899258D221410C4D84AE2CA9D98676
:1004C00021B30542104D848E21AA4449944C9528AD
:1004D000890605430B4D849E25137B4B1600441261
:1004E0004D848E21AA4449944449944449342800B7
:1004F000450B4D848E637148C2E220460B4D848EBD
:10050000637148C24600470C4D849E25139B362DCF
:100510005900480B4D848ECC6D1832B7004909CB79
:10052000848E25EACB004A0B4D84AE2DEC258A241F
:10053000004B0E4D848ECC9494B424AA645A004C83
:10054000094D848EB01F07014D0D4D848E4C5B9676
:10055000444934B7004E0D4D848E6C9A944449A49E
:100560009B164F0A4D849E25F35BB200500C4D84C0
:100570008E21C96C83123602510A557C9E25F34B9D
:10058000650D520E4D848E21C96C8352AA645A00A7
:10059000530C4D849E2513D335D4920554094D84B4
:1005A0008E410AFB0955094D848ECCDF9205560E0B
:1005B0004D848ECC2D29255192851100570D4D84E7
:1005C0008ECC4BA2244AA27401580E4D848E4C4B03
:1005D0004A495689929A16590C4D848E4C4B4A4979
:1005E0001676025A0D4D848E41CCC2AC988583009C
:1005F0005B09DB7C8E21EA4F035C0B4D848E300D52
:10060000D3621A065D09DB7C8EA93F0D015E081DD1
:10061000B4AE2CA9055F060D7C8E41600612C58E16
:1006200028610B35849E351934495102620C4D8482
:100630008EB0382499DBA000630A35849E25136BA5
:10064000C902640B4D84CE9641734B8600650C3510
:10065000849E251B86304B1600660C4D842EA912F5
:10066000664314B601670D45749E25B32543A8253E
:100670000B00680A4D848EB0C5A4B9056908C3840F
:100680009E50EA326A0B5474BE586B93A444016BBB
:100690000D4D848EB02929694954C9026C08CB8458
:1006A0000EA95F066D0D35840EA54549944449B4E5
:1006B000006E0935848EC4A4B9056F0A35849E2561
:1006C000734B1600700C45748E21C96C8312160191
:1006D000710B45749E41B32543D800720935848E51
:1006E000C4243602730C35849E254BD4244B16004B
:1006F000740C45849E301BA2B029520075093584C4
:100700008ECC93A204760B35848ECC9694922C02D8
:10071000770B35848ECC922889D205780B35848E60
:100720002CA98559520B790C45748ECC4951422D18
:1007300059007A0935848E41EB38087B0B5D7C3E8D
:10074000296C52C356017C0649858E077D0B5D7C62
:100750000E356C95C2260D7E091DB49E4849A40431
:1007600000000004FFFF05910793749E06059208A0
:1007700015BCAE5A0005930822BD1E490105940719
:1007800019BD8E240595099BBC8E444A0205960727
:1007900012758E280597099BBC9E64490005980A2E
:1007A0001DBC9E4849A4040599081ABC8E28090559
:1007B0009A071A761E29059C081BBD9E2902059DD5
:1007C000081ABE1E2501059E0B2CB59E2852DA1272
:1007D00000059F0A25B49E7E4A120005A00923B594
:1007E0009E4E090005A10A1CBC9E6489120005A347
:1007F000079374AE2105A4079A741E2905A5071254
:10080000751E0505A60915749E484A0005A8089A94
:10081000BC8E280905A90923B49E4E090005AA0823
:1008200093748EA40205AB079ABC1E2905AC089BE5
:10083000BCAE680805AD0712768E2805AF089BBCD4
:100840009E2E0005B00719758E2405B1091D748E02
:10085000A41C0505B2081D74CE210E05B3091D7434
:10086000CE218B0205B40709758E0005B5078B7480
:100870008E2405B60915748E2C8A0005B7078B7473
:100880008E0105B80893748E250105B90789BC8EC1
:100890000005BB081D748EB80005BC07099D8E00BD
:1008A00005BD0711750E0105BE078CAC8E2105BF75
:1008B000078BBC8E0105C00731858E0305C1070972
:1008C000BE8E0005C20709BC8E0005C30731850E28
:1008D0004905C40709BD8E0005D00C35848EA8C516
:1008E0009464530005D10A35848E21EC320805D278
:1008F0000BB4848EB01625520005D30A35848E4180
:100900000BBB0005D40B35848E410C355B0005D53F
:100910000832850EA50705D60B35848E410AD3B063
:100920000205D70F35848E41899228899228890241
:1009300005D80D35848E68499444D3860105D908BD
:100940001A9D0EA50005DA0945748E41EC0705DBFA
:100950000B35848E416C1C140005DC0C4D848EB06C
:1009600038886D910405DD0F35848E418992288980
:100970009228190205DE0B35848E28E9A459060554
:10098000DF0842750EA51F05E009B4842EAD6D1079
:1009900005E10E35848E418992288992920405E200
:1009A0000F35840E45899228899268500005E30D21
:1009B00045748E4189922889C20E05E40D35848ED6
:1009C000418992280C070505E50D45748EA8254A36
:1009D0004A5A580305E60B35848EA84B960E03053C
:1009E000E70C45748E41D45C94300405E8093584E5
:1009F0008E210D3B05E90F35848E245112251912E5
:100A00006D500005EA0E35848E41899228899268DE
:100A10000A05F00F35840E458992288992288902AB
:100A200005F10B35840E458992286C05F20A1D9C50
:100A30000E4589922805F30712A51E0505F4091530
:100A4000A49E484A00FB1D082A8D0EA516FB1E0910
:100A500015C48E2C5900FB1F0C2D8C0E4589922835
:100A60001D04FB200E35848E488992A8122583022E
:100A7000FB210C35848EA8C594645300FB220A35F3
:100A8000848E410BBB00FB230B35848E410C355B00
:100A900000FB240B35848E416C1C1400FB250C4D8F
:100AA000848EB038886D9104FB260F35848E418981
:100AB00092288992281902FB270935848E210D3B43
:100AC000FB280E35848E418992288992680AFB2979
:100AD000091D84AE301A04FB2A104584BE3849949F
:100AE000444986441B1400FB2B1045848E1C4A127B
:100AF00025519221D10605FB2C0F4584BE3849941F
:100B00004419166D5000FB2D1045848E1C4A122589
:100B10005186451B1400FB2E0D457C8EA8C59464A0
:100B200053BC00FB2F0E4D748EA8C5946453BC4576
:100B300000FB300E45748EA8C59464530E4400FB30
:100B4000310C35848E218C92B03208FB320B358407
:100B50009EB412654929FB330C35848E410BA324C6
:100B6000AC00FB340C35848E410C9544D302FB352C
:100B70000AB3841E2952A202FB360D35848E410A27
:100B8000D328091300FB380C35848E6853124D1B93
:100B900006FB39089B9C1E4909FB3A0B45748E41A4
:100BA0002C256107FB3B0D35848E414CA2301C1473
:100BB00000FB3C0E4D848EB038884914669104FBCE
:100BC0003E0D35848E448A3425D19401FB400BB40C
:100BD000842E2DA9658300FB410C35848E9B926881
:100BE000523201FB430C45749E41D3A224EC00FB1E
:100BF000440C35849E41538AE1A000FB460B3584AA
:100C00008EA88B940E03FB470E45748E415412CD73
:100C1000A2842100FB480B35848E218D92B001FB0C
:100C2000490E35848E2451126558B44101FB4A0E99
:100C300035848E418992448992680AFB4B0942852A
:100C40008E4CE901FB4C0B45849E7908BB0C02FBE2
:100C50004D0B45849E79101B0705FB4E0D45849E68
:100C60001D18342D0C0705FB4F0D4D848EB0A9C502
:100C7000946453000000672711241FBECFEFD8E013
:100C8000DEBFCDBF14E0A0E0B1E0E2E3F3E702C0D5
:100C900005900D92AE32B107D9F726E0AEE2B4E08E
:100CA00001C01D92AE3BB207E1F716E0CCE3D6E0FF
:100CB00004C02197FE010E940134CB33D107C9F74C
:100CC0000E9494280C9497390C940000662329F014
:100CD0006A3019F0862F90E008958FEF9FEF089506
:100CE00080E0089580E00895982F2091700581E0BC
:100CF000213208F043C080914C058111FCCF8091D6
:100D00006F0532E030934C0590934B059FEF909325
:100D10004A051092490520934805AFE4B5E0E8E2A2
:100D2000F5E090E0291331C0109227059091270536
:100D3000880F892B8093270580912605813049F5FE
:100D400010922605809127058093BB008091BC00FE
:100D500083FDF8CF85EC8093BC0080914C058230F8
:100D6000E1F380914A058F3FB1F080914A058032CE
:100D7000A1F080914A05803391F084E010924E05F5
:100D80001092700510924D0508953D9131939F5F2B
:100D9000C9CF85EEE0CF80E0F1CF82E0EFCF83E0F6
:100DA000EDCF8091040590910505891B990B08955D
:100DB0002F923F924F925F926F927F928F929F926B
:100DC000AF92BF92CF92DF92EF92FF920F931F9359
:100DD000CF93DF93CDB7DEB76C970FB6F894DEBF35
:100DE0000FBECDBF522E3D874E87252E462E372E65
:100DF000782E692EA982BF86C88AD98AEA8AFB8A98
:100E00000C8B1D8B988E8F8A21150CEA300703E21C
:100E100040070CEF500706E060077105810591055A
:100E200009F098F52F3F10EE310715EF410715E057
:100E30005107610571058105910509F008F40BC1A1
:100E40002F3F354D41415E47634071058105910556
:100E500009F008F40BC129813F85488959896A89BD
:100E60007B898C899D89A0E0992493940E94853583
:100E7000C9F4F1E0FE8B04E0802E912CA12CB12C62
:100E800089869A86AB86BC8616C1512CBCEABD8782
:100E9000E3E2EE878CEF282E96E0492E312C712C60
:100EA000612CD9CFA52CBD84CE84D22CE42CF32C7C
:100EB000072D162D29813F85488959896A897B89A3
:100EC0008C899D890E94D03429873A874B875C871B
:100ED00029853A854B855C85B6E0AB2EB12C263052
:100EE00031054105510568F089859A85AB85BC853A
:100EF00089309740A105B105E0F0F8E0AF2EA7E0FA
:100F0000BA2EC12CD12CE12CF12C00E010E029816B
:100F10003F85488959896A897B898C899D890E9486
:100F2000D034522E3D874E87252E462E372E782ED2
:100F3000692EA52CBD84CE84D22CE42CF32C072D55
:100F4000162D29813F85488959896A897B898C8931
:100F50009D890E94CE34AA24AA94BB24BA94EFE0BF
:100F6000CE2ED12CE12CF12C00E010E00E941A349E
:100F7000A52CBD84CE84D22CE42CF32C072D162D69
:100F80000E94D034A32FF42FE52F422F5A2F6F2F1A
:100F90007E2FCC24CA94DC2C8FE0E82EF12C411556
:100FA00051056105710521F4C12CD12C7601C39442
:100FB000AA24A3949A1409F4E5C001E00E8BCB0196
:100FC000BA0137E0660F771F881F991F3A95D1F74E
:100FD000A70196010E94DF33298F3A8F4B8F5C8FD8
:100FE00089849A84AB84BC8447E0880C991CAA1C31
:100FF000BB1C4A95D1F79501840112502109310992
:1010000048015901298D3A8D4B8D5C8D280D391D74
:101010004A1D5B1DAF89B88D2D933D934D935C9315
:101020001397FD0164837583868397831896CD9209
:10103000DD92ED92FC921B978E88882009F481C086
:1010400059829D849F86AE84A88A298A4A8A3B8ACF
:101050007C8A6D8A76C0512C01EE0D8715EF1E87B4
:1010600025E0222E412C312C712C612C29813F85C9
:10107000488959896A897B898C899D89A0E0912C4E
:101080000E94853509F00ECFA52CBD84CE84D22CCC
:10109000E42CF32C072D162D20E030EB4EE850EF1A
:1010A0006BE170E080E090E00E94D03429873A87BD
:1010B0004B875C871E8A89849A84AB84BC84A50193
:1010C000940160E070E0CB01A52CBD84CE84D22CCD
:1010D000E42CF32C072D162D29833A834B835C8354
:1010E0006D837E838F83988760E070E080E090E07E
:1010F0000E941A3429833F87488B598B6A8B7B8BDC
:101100008C8B9D8B0E89C12CD12C7601C39440E031
:1011100050E0BA01013009F052CFAF89B88D1D926D
:101120001D921D921C921397FD0114821582168246
:10113000178281E090E0A0E0B0E080879187A287ED
:10114000B38729813F85488959896A897B898C8938
:101150009D896C960FB6F894DEBF0FBECDBFDF91B0
:10116000CF911F910F91FF90EF90DF90CF90BF90A4
:10117000AF909F908F907F906F905F904F903F9037
:101180002F900895AF89B88D1D921D921D921C92CB
:101190001397FD01148215821682178281E090E078
:1011A000A0E0B0E080879187A287B3875982FD8550
:1011B000FF878E84888A49CFDF92EF92FF920F9348
:1011C0001F93CF93DF93FC01E080F18002811381B4
:1011D000D481C581B681D7809701A8016D2F7C2F5E
:1011E0008B2F9D2D35534C4051096109710981099F
:1011F00091092F3F34434C4051056105710581052C
:10120000910509F0D0F49701A8016D2F7C2F8B2F49
:101210009D2D07E00E943D35208331834283538317
:10122000648375838683978387E0DF91CF911F91D5
:101230000F91FF90EF90DF9008959701A8016D2F17
:101240007C2F8B2F9D2D3A56484151096109710918
:10125000810991092F3F39464841510561057105C2
:101260008105910509F098F49701A8016D2F7C2F55
:101270008B2F9D2D06E00E943D35208331834283D4
:101280005383648375838683978386E0CECF9701EB
:10129000A8016D2F7C2F8B2F9D2D345D404351096C
:1012A00061097109810991092F3F334D404351056F
:1012B000610571058105910509F098F49701A80170
:1012C0006D2F7C2F8B2F9D2D05E00E943D352083B7
:1012D000318342835383648375838683978385E058
:1012E000A4CF9701A8016D2F7C2F8B2F9D2D385AED
:1012F0004146510961097109810991092F3F374A16
:1013000041465105610571058105910509F098F483
:101310009701A8016D2F7C2F8B2F9D2D04E00E943B
:101320003D35208331834283538364837583868371
:10133000978384E07ACF9701A8016D2F7C2F8B2FA4
:101340009D2D3055434C510961097109810991095D
:101350002F3F3F44434C51056105710581059105BF
:1013600009F098F49701A8016D2F7C2F8B2F9D2DEC
:1013700003E00E943D35208331834283538364839D
:1013800075838683978383E050CF9701A8016D2FE3
:101390007C2F8B2F9D2D305A464851406109710991
:1013A000810991092F3F3F49464851406105710528
:1013B0008105910509F098F49701A8016D2F7C2F04
:1013C0008B2F9D2D02E00E943D3520833183428387
:1013D0005383648375838683978382E026CF970146
:1013E000A8016D2F7C2F8B2F9D2D30544D405340E5
:1013F00061097109810991092F3F3F434D405340D5
:10140000610571058105910509F098F49701A8011E
:101410006D2F7C2F8B2F9D2D01E00E943D35208369
:10142000318342835383648375838683978381E00A
:10143000FCCE80E0FACE809373060895CF93DF93BD
:10144000CDEFD5E08FE592E09CAF8BAF81E096E0E9
:101450000E94DC0DEBADFCAD0280F381E02D81E05C
:1014600096E0DF91CF9109949B01DC011896ED91F4
:10147000FC9141E067E10994833081F028F48130E8
:1014800099F08230A9F008958730A9F08830C9F02A
:101490008430B1F4809180008F7D03C08091800002
:1014A0008F7780938000089584B58F7784BD0895E9
:1014B00084B58F7DFBCF8091B0008F778093B00093
:1014C00008958091B0008F7DF9CFCF93DF93282FBF
:1014D00030E0F901E75DFC4F8491F901EB5EFC4FD0
:1014E000D491F901EF5FFC4FC491CC23A1F081119D
:1014F0000E943C0AEC2FF0E0EE0FFF1FE950FD4F79
:10150000A591B491EC91ED2381E090E009F480E0A5
:10151000DF91CF91089580E090E0FACF1F93CF93B1
:10152000DF93282F30E0F901E75DFC4F8491F9014A
:10153000EB5EFC4FD491F901EF5FFC4FC491CC23DB
:10154000A9F0162F81110E943C0AEC2FF0E0EE0F5B
:10155000FF1FE351FD4FA591B4918FB7F894EC9123
:10156000111108C0D095DE23DC938FBFDF91CF919E
:101570001F910895DE2BF8CFCF93DF9390E0FC010D
:10158000EB5EFC4F24918F5F9C4FFC01849188237C
:10159000C9F090E0880F991FFC01ED51FD4FA59116
:1015A000B491FC01E351FD4FC591D49161110DC07F
:1015B0009FB7F8948C91209582238C93888128235F
:1015C00028839FBFDF91CF910895623051F49FB778
:1015D000F8943C91822F809583238C93E8812E2B65
:1015E000EFCF8FB7F894EC912E2B2C938FBFEACFCF
:1015F0008E50806480937C0080917A008064809318
:101600007A0080917A0086FDFCCF809178009091DD
:10161000790008953FB7F8948091B8049091B90487
:10162000A091BA04B091BB0426B5A89B05C02F3F7A
:1016300019F00196A11DB11D3FBFBA2FA92F982FF8
:101640008827BC01CD01620F711D811D911D42E0F3
:10165000660F771F881F991F4A95D1F708958F92BB
:101660009F92AF92BF92CF92DF92EF92FF926B0167
:101670007C010E940A0B4B015C01C114D104E104FE
:10168000F104B9F00E940A0B681979098A099B09CB
:10169000683E73408105910580F321E0C21AD108AC
:1016A000E108F10888EE880E83E0981EA11CB11CA9
:1016B000E4CFFF90EF90DF90CF90BF90AF909F90DE
:1016C0008F900895009749F0FC0181E09191992352
:1016D00029F09A30D9F78F5FF9CF80E00895DC01C7
:1016E0001A96ED91FC9130E020E00994DC01169609
:1016F000ED91FC9130E020E040E069E10994DC01EB
:101700001696ED91FC9130E020E040E068E109940C
:101710009A01DC011696ED91FC91462F67E1099440
:10172000EF92FF920F931F93CF93DF931F92CDB74A
:10173000DEB77C018B01D8016C91673129F150F43F
:101740006531A0F40F90DF91CF911F910F91FF9021
:10175000EF9008956A3118F16E3FA1F7F8014181C9
:10176000498369E2C7010E946F0B0BC0F8014181F8
:101770004983D7011696ED91FC9130E020E0C70136
:1017800009950E5F1F4FD7CFF80181818983AE0184
:101790004F5F5F4F61E0C7010E94880BF2CF0F5F80
:1017A0001F4FD7011696ED91FC9130E020E040E00C
:1017B000C7010995C0CF462FDC011696ED91FC912B
:1017C00030E020E066E10994462FDC011696ED91A9
:1017D000FC9130E020E065E10994EF92FF920F93D5
:1017E0001F93CF93DF93EC01042F79016D3009F43F
:1017F00046C050F46B30C9F1693009F49FC06A30BB
:1018000009F465C080E05CC06E3009F44BC06F30F5
:1018100099F70E947F0BF7011381110F110F110F20
:101820006C89160F60E4CE010E94E40B612F629573
:101830006F706061CE010E94E40B612F6F70CE016A
:101840000E94DB0BF7016481606BCE010E94DB0B11
:10185000F701408151816281660F660F660FCE01EC
:101860000E94880B0150A1F727C061EF71E044236B
:1018700011F06CEE71E0CE010E94900B20C041117E
:1018800009C065EE71E00E94900BE881F9818289C0
:101890008C8B15C06EED71E00E94900BE881F98190
:1018A0008389F6CF0E947F0B61E8CE010E94E40B92
:1018B000602FCE010E94DB0BCE010E94760B81E0EF
:1018C000DF91CF911F910F91FF90EF900895EA85DE
:1018D000FB8530E020E040E068E2CE010995EE8132
:1018E000FF8130E020E040E064E1CE01099541E075
:1018F0006BE4CE010E946F0BE881F981448169E2BB
:10190000CE010E946F0B40E06BE4CE010E946F0B92
:10191000E881F981448169E2CE010E946F0B41E0C8
:101920006BE4CE010E946F0BE881F981458169E289
:10193000CE010E946F0B66EF71E09DCF8BE292E0CB
:101940009983888382E0A4CFCF93DF931F92CDB792
:10195000DEB76983BE016F5F7F4F0E94340A0F902C
:10196000DF91CF910895462FDC011896ED91FC91FF
:1019700030E020E060E20994EF92FF920F931F9312
:10198000CF93DF938C01C62FD42F7901673130F4C8
:101990006531B8F4643131F080E01BC0673101F18A
:1019A0006A31D0F7D8011896ED91FC9197014D2F2F
:1019B0006C2FC801DF91CF911F910F91FF90EF9095
:1019C000099460E00E94B30C6D2FC8010E94A40C22
:1019D00081E0DF91CF911F910F91FF90EF900895DB
:1019E00061E00E94B30CDECFFC016623D9F16A30BE
:1019F000C9F1818D811125C06C3F48F085E0818F50
:101A0000617070E0738B628B2EEF3FEF29C0683FEF
:101A100020F084E0818F6370F4CF603F20F083E09A
:101A2000818F6770EECF603E20F082E0818F6F7013
:101A3000E8CF262F30E0603C98F081E0818F6F7115
:101A4000E0CF8150818F2289338996E0220F331FA6
:101A50009A95E1F76F73262B338B228B8111D4CFAC
:101A6000C90108952FEF3FEFFBCF0F93DC01FC017D
:101A7000ED5BFF4F9081941B492F31979081961B0E
:101A8000692F01110EC04150621BDF968C91DF97C8
:101A9000481BD596ED91FC91D697CD0109950F91F4
:101AA0000895013091F76150421BEFCF0F93DC0195
:101AB000DF963C91DF97431BD596ED91FC910995FC
:101AC0000F910895FC01EC5BFF4F10823196DC0111
:101AD000AE5BBF4F2C9120833196108211962C91D2
:101AE00012973C91231718F0422F431B4083FC01AF
:101AF000E95BFF4F805C9F4FDC018C91281B2083AA
:101B00000895FC01EC5BFF4F10823196DC01AE5B67
:101B1000BF4F2C912083319612972C9120833196C0
:101B20008F5B9F4FDC018C9180830895CF93DF936F
:101B3000FC01A081B18183AD982F990F990F990F66
:101B400096AF50969C915097903208F09FE1990F74
:101B5000990F990F95AF24AD922F990F990F990F67
:101B600097AF51963C915197682F620F7727771F57
:101B70003617170614F4832F821BEF01C05CDF4F6A
:101B800098832196880F880F880F890F8883219664
:101B900080EF888354968D919C915597813F910554
:101BA00008F48883ED5BFF4F56968C918083DF911C
:101BB000CF9108950C94960D0C94960DCF93DF93CE
:101BC000342F3770E1E0F0E0DF0102C0AA0FBB1F45
:101BD0003A95E2F79D0150E0487FEC01E9ADFAAD9E
:101BE000A881B98150967C91749FD001759FB00DEA
:101BF00011246A0F7B2F711DE60FF71FDC01AE5811
:101C0000BF4F8C91823018F48081822B80838C911D
:101C1000813019F0808128272083DF91CF910895AA
:101C2000EF92FF920F931F93CF93DF937C01162FB8
:101C3000D42F011111C0C62FC20F4D2F612FC70124
:101C40000E94DE0D1F5FC113F8CFDF91CF911F916E
:101C50000F91FF90EF900895C22FC40F4D2F612F69
:101C6000C7010E94DE0DDF5FDC13F8CFEECF0F93CC
:101C7000DC01222371F1FC0101112DC0EA5BFF4F51
:101C80008081481730F131968081481710F53297DE
:101C9000908131978081260F2617C8F46917B0F418
:101CA0002FEF290F8217A8F4681708F4682F291757
:101CB00008F4922F961BD796ED91FC91D89704804B
:101CC000F581E02D292FCD01099503C0682F6917F3
:101CD00048F30F910895EC5BFF4F80816817C8F3BC
:101CE000319680816817A8F732969081319780816C
:101CF000240F241778F4491760F42FEF290F821767
:101D000040F7481708F4482F291708F4922F941B1E
:101D1000D2CF482F4917E8F6F2CFFC01E85BFF4F1E
:101D200020813181295E3F4F6F3F710509F010F529
:101D300061367105A0F085599F4FFC01808191812A
:101D4000280F391FC9010196FC014491442391F0E9
:101D5000F90144914617170641F40196089561343C
:101D6000710580F387599F4FE8CFFC018491280FBC
:101D7000311DE8CF90E080E00895DC0118964C9189
:101D80001897ED91FC911197249130E0042E02C038
:101D9000359527950A94E2F7842F860F883068F0EE
:101DA00031961196FC93EE93E49198E0941B01C058
:101DB000EE0F9A95EAF72E2B885018968C938FEF9A
:101DC0009FEF01C0880F6A95EAF7809582230895F6
:101DD0000F931F93CF93DF938C01EC01C45BDF4F14
:101DE000798368831886FC01E45AFF4F6081CE0135
:101DF0000E94BD0E8E83F801E35AFF4F6081CE0131
:101E00000E94BD0E8F83F801EE58FF4F90819A8794
:101E100081E0911180E08B87DF91CF911F910F912D
:101E20000895CF93C62F0E94BD0EC15021E030E02F
:101E300001C0220FCA95EAF7821BCF9108950F9334
:101E40001F93CF93DF931092530610921A068C01C2
:101E5000D0E0C0E0F80161918F01E0910306F091BC
:101E6000040681E096E009958F3F980749F18E3F7F
:101E70002FEF920779F3BC0181E096E00E948D0E6E
:101E80000097E1F0BC0181E096E00E94E80E6091CD
:101E90005F068DE496E00E94110F809371066091B9
:101EA00060068DE496E00E94110F609161068DE45A
:101EB00096E00E94110FD82FC80FCCCF80E0FBCF47
:101EC00080915306882329F090917106890FC80FDD
:101ED000CD1B8C2FDF91CF911F910F910895FC01A5
:101EE000E60FF11D849190E0982F88273196E491B8
:101EF0008E0F911D0895CF93DF9320914906309165
:101F00004A062817390709F488C0EC0190934A065D
:101F100080934906FC018491809359063196E4919F
:101F2000E0935A06FE013296E491E0935B06FE01CF
:101F30003396E491E0935C06FE013496E491E093DD
:101F40005D06FE013596E491E0935E06FE0136964D
:101F5000E491E0935F06FE013796E491E09360061A
:101F6000FE013896E491E0936106FE013996E49112
:101F7000E0936206FE013A96E491E0936306FE0167
:101F80003B96E491E0936406FE013C96E491E09375
:101F90006506FE013D96E491E0936606FE013E96DD
:101FA000E491E0936706FE013F96E491E0936806B2
:101FB000FE017096E491E093690661E1CE010E9412
:101FC0006F0F90936B0680936A0663E1CE010E94C7
:101FD0006F0F90936D0680936C06809149069091E7
:101FE0004A06892BD1F08091660680936F06409156
:101FF00067064093700690916E06992371F09130B8
:1020000079F490916806891714F490936F06809183
:102010006906841714F480937006DF91CF910895B8
:102020003091630620916506082E000C990B622FF3
:10203000022E000C770B630F711D37FD7A95861702
:1020400097071CF4320F30936F06241734F7209350
:102050007006E3CFCF93DF93EC016CAFEFA9F8AD3F
:102060000190F081E02D0995EFA9F8AD0280F38190
:10207000E02DCE01DF91CF910994AF92BF92CF9224
:10208000DF92EF92FF920F931F93CF93DF9300D0D5
:1020900000D01F92CDB7DEB78C01DC01DB96AC908F
:1020A000DB97DC96EC90DC97ED91FC91B188FE2CEF
:1020B000D12CC12CD801ED91FC9111978089D99632
:1020C0002D913C911C82FD828B83B8E08B9FC001D7
:1020D00011248C9DA0018D9D500D9C9D500D1124AF
:1020E000240F351F3A832983D8011496ED91FC9172
:1020F0009E012F5F3F4F41E06FE0C8010995F394C7
:102100008F2D8E198A1528F4BFEFCB1ADB0AFB142A
:1021100088F20F900F900F900F900F90DF91CF915A
:102120001F910F91FF90EF90DF90CF90BF90AF90F5
:102130000895DF92EF92FF920F931F93CF93DF9357
:102140007C01D62F142FD22EC02F00E00E94370E14
:1021500001E02C2F412F6D2FC7010E94370E6FEF2A
:102160006D0D6D0F2C2F412FC7010E94370E4FEFC1
:102170004C0F410F00E02D2D6D2FC7010E94370E2F
:10218000DF91CF911F910F91FF90EF90DF90089515
:102190000F931F93CF93DF938C01C62F642FCC3204
:1021A000E8F4CA3208F041C0C83271F1C93209F40A
:1021B00042C080E0C034D0F1CF73F801EC0FF11DC4
:1021C000878D8F3F91F1C031E0F00E94650A21E0D8
:1021D000892B09F420E0F801228F27C0CD3289F144
:1021E00040F384EB8C0F823020F7CF73C00FD12FD8
:1021F000D11D8F8D411133C061E00E94BC0A60E0A7
:102200008F8D0E948E0A11C0015E1F4FD0E0F80131
:1022100081918F018F3F31F061E0D03108F062E0B1
:102220000E94BC0ADF5FD63191F781E0DF91CF9148
:102230001F910F91089570E090E080E00E942F0BB5
:10224000F4CF85E090E0433010F082E090E0880F1A
:10225000991F880F991F05970197F1F7E6CF62E064
:102260000E94BC0AE2CF85ED8093BC008091BC0047
:1022700084FDFCCF10924C05089520918D04260F0B
:102280003327331F21323105ECF420914C05FC013A
:1022900090E080E0243069F082E00895A0918D0400
:1022A0002191AC0145595B4FA40FB52FB11D2C9363
:1022B0000196861798F380918D04680F60938D04C2
:1022C00080E0089581E00895089508950895E091CB
:1022D000050580910405E81730F4F0E0EA5FFA4F55
:1022E000808190E008958FEF9FEF0895909105050C
:1022F000809104052FEF3FEF981748F4E92FF0E0A5
:10230000EA5FFA4F208130E09F5F90930505C90195
:102310000895CF92DF92EF92FF920F931F93CF9386
:10232000DF937C01CB018A0120914D05222389F0A6
:10233000EB016B01C40ED51ECC15DD0569F069916A
:10234000D701ED91FC910190F081E02DC701099535
:10235000F3CF642F0E943D11C801DF91CF911F91EF
:102360000F91FF90EF90DF90CF900895CF93DF9380
:102370001F92CDB7DEB7698320914D052223F9F076
:1023800020917005203258F021E030E0FC013383C9
:10239000228390E080E00F90DF91CF9108958091AB
:1023A0004E05E82FF0E0E15BFA4F998190838F5F53
:1023B00080934E058093700581E090E0ECCF61E062
:1023C000CE0101960E943D11F7CFCF93C62F91E029
:1023D00090934D0590E690936F0510924E051092E4
:1023E0007005682F81E795E00E94B6116C2F81E798
:1023F00095E00E94B61181E0CF910C9474060F9382
:102400001F93CF93DF938B0191E090934D0590E65E
:1024100090936F0510924E0510927005682F81E71A
:1024200095E00E94B611E801085F1F4F699181E7AE
:1024300095E00E94B611C017D107C1F781E0DF9186
:10244000CF911F910F910C9474068EE00E94F80AB0
:10245000BC01990F880B990B0E94C4322091FC0497
:102460003091FD044091FE045091FF040E945233CC
:1024700020E030E040E85AE30E9452336093670462
:10248000709368048093690490936A04089580911E
:10249000C10481111092C10408958091D504E82FE0
:1024A000F0E0EE5AFB4F9091E7049083E1E0E80FF3
:1024B000F0E0EE5AFB4F9091E8049083E2E0E80FE1
:1024C000F0E0EE5AFB4F9091EF0490839091E90475
:1024D000E3E0E80FF0E0EE5AFB4FA92FB0E0A75F72
:1024E000BE4F2C912083E4E0E80FF0E0EE5AFB4F62
:1024F00090838B5F8093D5040895CF92DF92EF9203
:10250000FF920F931F93CF93DF936C01EB017B013D
:10251000E40EF51E10E000E0CE15DF0561F06991D4
:10252000D601ED91FC910190F081E02DC601099555
:10253000080F191FF1CFC801DF91CF911F910F91A3
:10254000FF90EF90DF90CF900895089590E080E0A5
:102550000895CF93DF9391E090934D0590E690938B
:102560006F0510924E0510927005682F81E795E077
:102570000E94B61181E00E94740680914C05811181
:10258000FCCF81E080934C0510924B059FEF909318
:102590004A051092490510924805809327058091BD
:1025A0002705806C8093270580912605813061F591
:1025B00010922605809127058093BB008091BC0076
:1025C00083FDF8CF85EC8093BC0080914C05813071
:1025D000E1F380914905811119C080914905E8E234
:1025E000F5E0A6E0B5E0C0E0C81312C01092050502
:1025F000C093040580910505C81771F081E795E047
:102600000E947611D82FF6CF85EEDDCF81E0E7CF9F
:1026100091919D93CF5FE8CF8D2FDF91CF9108955A
:102620000F931F93CF938B01C0E1C80F8C2F0E9493
:10263000A912682F012B39F46F7D8C2FCF911F9138
:102640000F910C94E5116062F8CF1F93CF93DF9345
:10265000EB0110E1180F812F0E94A912682F6C7FE7
:10266000C230D10561F0C330D10559F0219709F48A
:102670006160812FDF91CF911F910C94E511626011
:10268000F8CF6360F6CF2F923F924F925F926F9296
:102690007F928F929F92AF92BF92CF92DF92EF92F2
:1026A000FF920F931F93CF93DF9300D01F92CDB76C
:1026B000DEB77C01845B9F4F9B838A83C7010E94A6
:1026C000E80EF701ED5AFF4F50803B9660818A81FA
:1026D0009B810E94110FD82EF701E15AFF4F6081B4
:1026E0008A819B810E94110F182FF701E05AFF4F3A
:1026F00060818A819B810E94110F8983EA81FB811D
:10270000868118160CF077C082818D0D82838381BB
:102710008519811B8383148215825701FAE5AF0E58
:10272000B11C47018BE5880E911C670192E7C90E29
:10273000D11CF50160818A819B810E94BD0E482ECB
:10274000F40160818A819B810E94BD0E382EEA814E
:10275000FB8114817580642CEA81FB812680211A1B
:10276000818581110FC0628143818385F601808359
:10277000222D621408F4262D470D610F00E0C701D9
:102780000E94370E621420F06218739410E0E4CFB8
:10279000160DEA81FB8114837582632CEA81FB812B
:1027A0002680211A628143818285F6018083222D51
:1027B000621408F4262D470D610F00E0C7010E9446
:1027C000370E621420F06218739410E0E7CF160DF4
:1027D000EA81FB811483758261E0CF010E94BD0E06
:1027E0008111B5CFEA81FB81858185150CF4A1CFDC
:1027F0008285F601808389810F900F900F90DF9181
:10280000CF911F910F91FF90EF90DF90CF90BF90ED
:10281000AF909F908F907F906F905F904F903F9080
:102820002F900895AF92BF92CF92DF92EF92FF92D6
:102830000F931F93CF93DF93EC018C010C5F1F4F1D
:10284000FC01E858FF4F0190F081E02DC801099587
:102850005C018EEFA8168FEFB80630F5FE01E55843
:10286000FF4FD0807E01EAE7EE0EF11CF701C08039
:10287000BC970190F081E02DC8010995FE01EE5A48
:10288000FF4FC082CD5ADF4F8D0D8883B501C8013F
:102890000E948D0E0097A9F0BC01C8010E9443134D
:1028A000F7019081890F808381E090E0DF91CF91E3
:1028B0001F910F91FF90EF90DF90CF90BF90AF905E
:1028C000089580E0EDCFDF92EF92FF920F931F9378
:1028D000CF93DF93082FD62E10921A06EA0110E04C
:1028E0006991E0910306F091040681E096E0099574
:1028F0007C018FEFE816F80611F18EEFE8168FEFE6
:10290000F80671F3E0914B06F0914C0681E096E0F9
:10291000099500934F068D0D80935006B70181E015
:1029200096E00E948D0E009741F0BC0181E096E098
:102930000E944313080F180FD3CF80E0FBCF812FE5
:10294000DF91CF911F910F91FF90EF90DF9008954D
:1029500026E636E030930406209303060C946314B5
:102960007F928F929F92AF92BF92CF92DF92EF921F
:10297000FF920F931F93CF93DF93D82F862E142FA0
:102980005901C02EE0914B06F0914C0681E096E093
:102990000995880E84EF9CE09093040680930306CB
:1029A000C5010E941F0FC82F912C811720F4912E72
:1029B000981A9694C12FF0906F06D82CDF1880914A
:1029C0007006F81A81E00E941B0A7D2C7F0C1D2DD9
:1029D000E11032C07D2E7C18CC2E1D2FDD1A171170
:1029E0002EC080E0E11001C081E00E941B0A84EF4C
:1029F0009CE09093040680930306A501682D8D2F1B
:102A0000890D0E94631481E0DF91CF911F910F9196
:102A1000FF90EF90DF90CF90BF90AF909F908F90FE
:102A20007F900C941B0A00E02C2F412F6D2F81E02A
:102A300096E00E94370E1F5F1711F5CFCBCF1150D4
:102A4000C394C3940F2D0C0D0C1B4D2D410F2C2D39
:102A5000612F81E096E00E949910C1CFEF920F9311
:102A6000CF93C0916F06CF5F90917006C91B01E0B4
:102A7000841300E0442361F0F90181E091919923EE
:102A800051F09F019A30D1F7481711F08F5FF6CFC0
:102A90002115310511F42DE134E0409143064250F7
:102AA000E02E81E00E94B0148C2FCF910F91EF9017
:102AB00008952F923F924F925F926F927F928F92E2
:102AC0009F92AF92BF92CF92DF92EF92FF920F93BD
:102AD0001F93CF93DF93CDB7DEB76A970FB6F89405
:102AE000DEBF0FBECDBF2F8B3987488F598F6A87C6
:102AF0007A8F1C011E8B0D8B6091B6067091B70604
:102B00008091B8069091B90624E630E040E050E0AC
:102B10000E947234522E632E742E852E962E788B40
:102B20008F87492E8091B0069091B106A091B20690
:102B3000B091B3066C017D01FF0CCC08DC2C760152
:102B40009C01AD016C2D7C2D8C2D9C2D0FE10E94E4
:102B50003D35A12CEAECBE2EFAE9CF2EABE3DA2EFE
:102B6000E12CF12C00E010E00E949F34A52CB62C43
:102B7000C72CD82CE92CF8880F85142D0E941A3404
:102B80000FE10E94583529833A834B835C836D8320
:102B90007E838F83988789819A81AB81BC81BB0FAB
:102BA000880B982FDC018B879C87AD87BE87252DEE
:102BB000362D472D582D692D7F2D8F85942DA98079
:102BC000BA80CB80DC80EB84FE2C0E2D1E2D0E9463
:102BD000733529833B874F87588B698B7A8B8B8B17
:102BE0009C8B8F889A8C282D3985488D598D6A85C4
:102BF000792DC1012115304B4E48504F6B41710565
:102C00008105910569F060F0812CB0EBB987EEE8A1
:102C1000E88FF0EFF98F8BE18A87912C212C312CF2
:102C2000282D3985488D598D6A85792DC101211549
:102C300038454744584F6D4071058105910560F452
:102C4000812CB8E5B987E7E4E88FF8EFF98F8DE0DC
:102C50008A87912C212C312CA980BB84CF84D888E1
:102C6000E988FA880B891C89282D3985488D598D6A
:102C70006A85792DC1010E94D03429013A011FE0F3
:102C8000A12E9FE0491651046104710440F0ABE5A8
:102C90004A16510461047104D0F0BAE5AB2EB12C90
:102CA000C12CD12CE12CF12C00E010E029813B85D6
:102CB0004F85588969897A898B899C890E941A3441
:102CC000822E3987488F598F6A87972E1C01A980D9
:102CD000BB84CF84D888E988FA880B891C89282D81
:102CE0003985488D598D6A85792DC1010E94CE3470
:102CF000AA24AA94BB24BA94AFE0CA2ED12CE12C0A
:102D0000F12C00E010E00E941A34A980BB84CF842B
:102D1000D888E988FA880B891C890E94D034C901B7
:102D2000DA01812C912C540183940097A105B105FF
:102D300031F088248A94982CEFE0AE2EB12CBC019F
:102D4000CD0127E0660F771F881F991F2A95D1F7BD
:102D5000A50194010E94DF33362E272E182F67E03D
:102D6000440C551C661C771C6A95D1F7B2E05B1ABF
:102D700061087108420E531E641E751E84E190E0C6
:102D80000E94B4359A838983FC0190828182862DCA
:102D900083708283538244827CE0B694A794979494
:102DA00087947A95D1F7F82DF07F8F2E812AA9810B
:102DB000BA8115968C92159716962C92169717969F
:102DC0003C921797ED89FE89BD018AE1EF2B19F03E
:102DD00069817A8182E20E94FF1189819A8100973C
:102DE000D1F06A960FB6F894DEBF0FBECDBFDF916B
:102DF000CF911F910F91FF90EF90DF90CF90BF90F8
:102E0000AF909F908F907F906F905F904F903F908A
:102E10002F900C9450366A960FB6F894DEBF0FBE12
:102E2000CDBFDF91CF911F910F91FF90EF90DF9079
:102E3000CF90BF90AF909F908F907F906F905F905A
:102E40004F903F902F9008952F923F924F925F9214
:102E50006F927F928F929F92AF92BF92CF92DF92AA
:102E6000EF92FF920F931F93CF93DF93CDB7DEB70F
:102E70002D970FB6F894DEBF0FBECDBF3C01C982BF
:102E8000DA82EB82FC820D831E832F833887498789
:102E90005A876B877C878AA18D873C2C2D2C9E2C92
:102EA000502E412EB22EC984DA84EB84FC8484E156
:102EB00090E00E94B4358C01FC01D082C182862D45
:102EC000880F880F880F845D0E94A912F92DF37076
:102ED0009F2E8C7F982AF8019282238234824CE0C4
:102EE000F694E794D794C7944A95D1F7FC2DF07FD8
:102EF000CF2E8B2D8F70C82AF801C582468257824B
:102F0000B80182E3F1E06F16710431F082E06816D7
:102F1000710409F44AC08AE20E94FF1130E1F32EE5
:102F2000F60C8F2D0E94A91291E0682FA9123FC0C4
:102F300060648F2D0E94E511E1E06E167104C9F105
:102F4000F2E06F167104D1F1A092AD062CE2F22EE0
:102F50008F2D0E94A91283789D8591118C60E0E1EC
:102F60008E9EB0011124682B8F2D0E94E511011552
:102F7000110549F1C8012D960FB6F894DEBF0FBEBA
:102F8000CDBFDF91CF911F910F91FF90EF90DF9018
:102F9000CF90BF90AF909F908F907F906F905F90F9
:102FA0004F903F902F900C9450368AE3B5CF6F7BB3
:102FB000C0CFA092AE0694E3F92ECACFA092AF067E
:102FC0008CE3F82EC5CF2D960FB6F894DEBF0FBE5A
:102FD000CDBFDF91CF911F910F91FF90EF90DF90C8
:102FE000CF90BF90AF909F908F907F906F905F90A9
:102FF0004F903F902F9008952F923F924F925F9263
:103000006F927F928F929F92AF92BF92CF92DF92F8
:10301000EF92FF920F931F93CF93DF93CDB7DEB75D
:10302000AA970FB6F894DEBF0FBECDBF622E298FD0
:10303000732E3A8F4B8F5C8F6D8F7E8F8F8F98A3FF
:1030400019A708A793012F3F34434C405105610550
:1030500071058105910509F050F4198E85E38A8F79
:103060008CE08B8F1C8E1D8E1E8E1F8E18A2298DBC
:103070003A8D4B8D5C8D6D8D7E8D8F8D98A1211538
:103080003C4A43425C4F664071058105910569F0F9
:1030900060F0198E8CEA8A8F83E28B8F8CEF8C8F95
:1030A00086E08D8F1E8E1F8E18A2CE0149960E943B
:1030B000DC088FA3798CBA8DAB8DFC8DED8D6E8C79
:1030C0005F8C48A0272D3B2F4A2F5F2F6E2F762D28
:1030D000852D942D2F3F05ED300701E140070EE7C8
:1030E000500703E0600771058105910511F008F0B4
:1030F0009EC0CE010D964C01A12CE4E0BE2EFBE655
:10310000CF2EA4EFDA2EB4E1EB2EF12C00E010E08C
:10311000852D942D0E94D806798D6A8D5B8D4C8DFE
:103120003D8D2E8D9F8D88A1E8A5F9A5E130F10593
:1031300009F445C0329709F45EC070939506609318
:1031400096065093970640939806309399062093DD
:103150009A0690939B0680939C0680E019A2412CCE
:10316000F4E0FAA30BE60BA314EF1CA394E19DA3D8
:10317000512C612C712C8F938FA0A82ECD84DE84CE
:10318000EF84F88809891A892B893C894D895E89E1
:103190006F89788D88A599A50E9424170F9099A111
:1031A000913009F0FBC08101242D3AA14BA15CA113
:1031B0006DA1752DC3010E94591519A2EFC070931E
:1031C0009D0660939E0650939F064093A006309301
:1031D000A1062093A2069093A3068093A40680E004
:1031E00019A2412CE4E0EAA3FBE6FBA304EF0CA345
:1031F00014E11DA3BDCF7093A5066093A60650935E
:10320000A7064093A8063093A9062093AA06909398
:10321000AB068093AC0680E019A2412C94E09AA3FF
:10322000EBE6EBA3F4EFFCA304E10DA3A1CFCE01E9
:103230000D964C01A12CB12CC12CD12CE12CF12CE0
:1032400000E010E0852D942D0E94D806298C3A8C40
:10325000BB8DAC8DFD8DEE8D08A519A50130110536
:1032600009F44EC00230110509F4A5C100E010E0D8
:1032700091014B2F5A2F6F2F7E2F8F8D98A10E9477
:10328000D806422E3AA34BA35CA36DA3572E3C0154
:1032900070E060E090E080E00E94101340928506AC
:1032A0009AA190938606EBA1E0938706FCA1F09388
:1032B00088060DA10093890650928A0660928B06BB
:1032C00070928C06898D809395068A8D80939606E0
:1032D0008B8D809397068C8D809398068D8D80932F
:1032E00099068E8D80939A068F8D80939B0688A178
:1032F00080939C0681E011E019A3312C212C3BCF57
:103300000F8D09A318A11EA31091B506123009F064
:1033100019C191014B2F5A2F6F2F7E2F802F9EA105
:1033200030584A41564061097109810991092F3786
:10333000304E42475849624071058105910509F0B8
:1033400008F446C02091A5063091A6064091A70634
:103350005091A8066091A9067091AA068091AB06CB
:103360009091AC065101CB2EDA2EEF2EFE2E09A144
:103370001EA10E947C3561F110929D0610929E065E
:1033800010929F061092A0061092A1061092A2061B
:103390001092A3061092A40611E019A389A1AA967F
:1033A0000FB6F894DEBF0FBECDBFDF91CF911F9156
:1033B0000F91FF90EF90DF90CF90BF90AF909F90D4
:1033C0008F907F906F905F904F903F902F900895D7
:1033D00040908D0680918E068AA390918F069BA3C4
:1033E000009190060CA3109191061DA35090920697
:1033F0006090930670909406CE010D964C01A42C1B
:10340000BAA0CBA0D02EE12EF52C830191014B2F39
:103410005A2F6F2F7E2F89A19EA10E94D80661E0AE
:1034200070E081E090E00E94101319A2298D3A8D7E
:103430004B8D5C8D6D8D7E8D8F8D98A130584A415E
:10344000564061097109810991092F37304E424771
:103450005849624071058105910509F008F4A7C03B
:1034600081E08093B5062091A5063091A606409193
:10347000A7065091A8066091A9067091AA068091AE
:10348000AB069091AC06A0E00E948535F1F185EA8B
:1034900096E00E94DC088FA3A0908D06B0908E0667
:1034A000C0908F06D0909006E0909106F090920622
:1034B00000919306109194062091A5063091A606DE
:1034C0004091A7065091A8066091A9067091AA069E
:1034D000CE0101964C018091AB069091AC060E9402
:1034E000D8061F928FA0A12CC980DA80EB80FC80C7
:1034F0000D811E812F81388549855A856B857C8594
:1035000082E090E00E9424170F90898D80939D06A1
:103510008A8D80939E068B8D80939F068C8D8093E1
:10352000A0068D8D8093A1068E8D8093A2068F8D2F
:103530008093A30688A18093A40681E0222423948B
:10354000312C19CE20938D0630938E0640938F0632
:103550005093900660939106709392068093930621
:10356000909394068E01035F1F4F4801A12CB12C4C
:10357000C12CD12CE12CF12C00E010E091014B2F5B
:103580005A2F6F2F7E2F89A19EA10E94D806422E0E
:103590003AA34BA35CA36DA3572E3C0161E070E0FE
:1035A00081E090E00E94101311E019A33FCF88E062
:1035B0008093B506AACF0091B50609A31F8D1EA35F
:1035C00008A10AA719A1113009F0F9C091014B2FE8
:1035D0005A2F6F2F7E2F8EA1902F30584A41564080
:1035E00061097109810991092F37304E42475849C5
:1035F000624071058105910561F158F12091A506A0
:103600003091A6064091A7065091A8066091A906A0
:103610007091AA068091AB069091AC065101CB2E19
:10362000DA2EEF2EFE2E0EA11AA50E947C3589F00F
:103630001092A5061092A6061092A7061092A80650
:103640001092A9061092AA061092AB061092AC0630
:10365000A5CE40908D0610918E061AA380918F06FC
:103660008BA3909190069CA3009191060DA350907E
:1036700092066090930670909406CE010D964C01D0
:10368000A42CB12ECBA0DCA0E02EF52C830191015F
:103690004B2F5A2F6F2F7E2F8EA19AA50E94D806EE
:1036A00061E070E082E090E00E94101319A2298D81
:1036B0003A8D4B8D5C8D6D8D7E8D8F8D98A13058A0
:1036C0004A41564061097109810991092F37304EED
:1036D00042475849624071058105910509F008F497
:1036E000A3C082E08093B50620919D0630919E068E
:1036F00040919F065091A0066091A1067091A2068C
:103700008091A3069091A406A0E00E948535F1F176
:103710008DE996E00E94DC088FA3A0908D06B09002
:103720008E06C0908F06D0909006E0909106F090A3
:103730009206009193061091940620919D06309177
:103740009E0640919F065091A0066091A10670913F
:10375000A206CE0101964C018091A3069091A40689
:103760000E94D8061F928FA0A12CC980DA80EB801E
:10377000FC800D811E812F81388549855A856B8596
:103780007C8581E090E00E9424170F90898D8093C2
:10379000A5068A8D8093A6068B8D8093A7068C8DB7
:1037A0008093A8068D8D8093A9068E8D8093AA069E
:1037B0008F8D8093AB0688A18093AC06BECE2093FC
:1037C0008D0630938E0640938F065093900660933B
:1037D00091067093920680939306909394068E01BF
:1037E000035F1F4F4801A12CB12CC12CD12CE12C1F
:1037F000F12C00E010E091014B2F5A2F6F2F7E2FFC
:103800008EA19AA50E94D806422E3AA34BA35CA390
:103810006DA3572E3C0161E070E082E090E00E94D1
:10382000101311E019A343CF88E08093B506AECF03
:10383000CF92DF92EF92FF920F931F93CF93DF937C
:103840008091EC04882309F402C1813009F408C195
:103850002FE7C21626E9D20628E9E206F10408F0AD
:1038600008C18091F4049091F504A091F604B09100
:10387000F7048093630490936404A0936504B09369
:1038800066048093F0049093F104A093F204B09343
:10389000F30460E085E00E948E0A81E08093ED04ED
:1038A000D701C60180589649A849B1098038944883
:1038B000AE41B10508F0FBC08091F8049091F90485
:1038C000A091FA04B091FB04809363049093640484
:1038D000A0936504B09366048093F0049093F10480
:1038E000A093F204B093F30461E081E10E948E0A98
:1038F00082E08093ED041091C804111118C08091EA
:10390000F4049091F504A091F604B091F70480932B
:10391000630490936404A0936504B0936604809359
:10392000F0049093F104A093F204B093F304809117
:10393000D3048823C1F08091F8049091F904A091F8
:10394000FA04B091FB048093630490936404A09301
:103950006504B09366048093F0049093F104A093FF
:10396000F204B093F3048091D204823009F4A4C02D
:10397000833009F4B9C0813061F48091F0049091F2
:10398000F104A091F204B091F304C80ED91EEA1E0E
:10399000FB1EC091ED04D0910001CD1751F061E004
:1039A0008CE00E948E0A64E670E080E090E00E9465
:1039B0002F0BC701B601112309F4B3C024E630E090
:1039C00040E050E00E94723410E000E00E94FC17DA
:1039D0008091F4049091F504A091F604B091F7045D
:1039E0008135934CA105B10508F4A0C083E00E9485
:1039F000A912682F6D7F83E00E94E5116091630436
:103A000070916404809165049091660424E630E02E
:103A100040E050E00E94723401E010E00E94FC1788
:103A2000CD1761F064E670E080E090E00E942F0B1B
:103A300060E08CE00E948E0AC0930001DF91CF917C
:103A40001F910F91FF90EF90DF90CF900895C0905D
:103A50000501D0900601E0900701F0900801F8CE32
:103A6000C090D604D090D704E090D804F090D90448
:103A7000EFCE8091F8049091F904A091FA04B091EE
:103A8000FB048093630490936404A0936504B09353
:103A900066048093F0049093F104A093F204B09331
:103AA000F30461E085E00E948E0A83E0F7CE60E0D7
:103AB00081E10E948E0A1FCF8091F0049091F10461
:103AC000A091F204B091F3048C159D05AE05BF05DD
:103AD00030F020E5C22E23ECD22EE12CF12CC81AB6
:103AE000D90AEA0AFB0A55CF8091F0049091F104BB
:103AF000A091F204B091F304C816D906EA06FB06B9
:103B000048F49C01AD012C193D094E095F0969017A
:103B10007A013FCF80E5C82E83ECD82EE12CF12C22
:103B200038CF64547D4F8F4F9F4F48CF83E00E9422
:103B3000A912682F626083E00E94E51171CF0F9394
:103B40001F9320910005309101054091020550918D
:103B50000305A4E6B0E00E9407346093B0067093BA
:103B6000B1068093B2069093B306109205051092A9
:103B7000040510924E051092700510924C0581E0DC
:103B800080934B051092260561E082E10E948E0A27
:103B900061E083E10E948E0AE9EBF0E080818E7F94
:103BA000808380818D7F808388E48093B80085E462
:103BB0008093BC0084E691E190938C0480938B0405
:103BC00085E691E19093900480938F0460EC87EBFD
:103BD0000E94E51160E880E10E94E51160E881E162
:103BE0000E94E51160E882E10E94E5116CE080E14D
:103BF0000E94E5116CE081E10E94E5116CE082E138
:103C00000E94E51160E281EB0E94E51160E881EB22
:103C10000E94E51110E000E020E034E04BE654EFB4
:103C200064E170E080E090E00E9459150E94181C49
:103C300070E060E090E080E00E94251370E060E0BA
:103C400081E090E01F910F910C9425130F931F9327
:103C500087E00E94650A892B11F583E00E94A91272
:103C6000682F6B7F83E00E94E511609105017091E0
:103C70000601809107019091080124E630E040E0C0
:103C800050E00E94723402E010E00E94FC1770E0E5
:103C900060E082E090E01F910F910C94251383E087
:103CA0000E94A912682F646083E01F910F910C9409
:103CB000E511CF93DF9380E190E00E94F431C0E002
:103CC000D5E0888381E190E00E94F431898382E12C
:103CD00090E00E94F4318A8383E190E00E94F43105
:103CE0008B83CE01DF91CF910895CF93DF9386E24E
:103CF00090E00E94F431CCEFD4E0888387E290E03A
:103D00000E94F431898388E290E00E94F4318A8332
:103D100089E290E00E94F4318B83CE01DF91CF9154
:103D200008950F931F93CF93DF9300EF14E0CCE23D
:103D3000D0E0CE010E94F431F80181938F012196E9
:103D4000C833D105B1F780EF94E0DF91CF911F9197
:103D50000F910895CF92DF92EF92FF920F931F93EE
:103D6000CF93DF93EB017B0124E0E20EF11C8B018A
:103D70006C01C61AD70AC601800F911F0E94F43148
:103D8000F80181938F01EE15FF05A9F7CE01DF91B0
:103D9000CF911F910F91FF90EF90DF90CF900895FA
:103DA0000C94F431FC01A081B18150962C9183AD2B
:103DB00038E0839FC0011124289FA001299F500D46
:103DC000112470E060E081AD92AD0C94D9361F9360
:103DD000CF93DF93EC010E943D101CAD8BAD180F0B
:103DE000E881F9818189181768F0EC81FD8130E064
:103DF00020E040E060E1CE01099580E0DF91CF91C5
:103E00001F910895FE01ED58FF4F8081882319F01E
:103E1000CE010E94D21E612FCE010E942A1081E0A5
:103E2000EDCFCF93DF93EC01FC01ED58FF4F808184
:103E3000882319F0CE010E94D21E60E0CE01DF91EE
:103E4000CF910C942A103F924F925F926F927F9283
:103E50008F929F92AF92BF92CF92DF92EF92FF929A
:103E60000F931F93CF93DF93982E892E162F5A010D
:103E7000C0916F06CF5F80917006C81B892D0E948C
:103E8000620B782E1111115080914406772009F4AD
:103E90005DC08350990B6C2F70E00E94CB33F62EDF
:103EA000F718C5010E94620B181710F01FEF180FCA
:103EB000C12ECF18C3941F1508F4C12C82E796E0D9
:103EC00090934C0680934B0681E096E00E94111F70
:103ED00044244394D0916F067720E9F03090430654
:103EE000892D982D0E94620B582E6D2ED12C5D10BD
:103EF00032C0C59DD00D112480917006442D481B01
:103F00004C1B4D0F00E02091430660E081E096E0FD
:103F10000E94370EDD5FD12CFD103AC081E096E0A3
:103F20000E94E71E8111D6CFDF91CF911F910F9193
:103F3000FF90EF90DF90CF90BF90AF909F908F90C9
:103F40007F906F905F904F903F9008956C2F0E94EC
:103F5000BF33F82EA6CF292D382DDD2079F0E92D9D
:103F6000F82D81E09191992339F09F019A30D1F792
:103F7000D81621F08F5FF6CF20E030E0E12C00E092
:103F8000432D662D80E00E94B0146C0ED394AFCF09
:103F90004C2D4D0D95016D2F812F0E942E15D80FA0
:103FA000D394BACF0F931F93CF93DF93EC01683173
:103FB00009F46EC058F46431F9F0F901673181F009
:103FC00080E0DF91CF911F910F910895693109F43D
:103FD0009CC06032A9F76AE4CE010E946F0B56C004
:103FE000442309F453C081918EBD00000DB407FE37
:103FF000FDCF8EB54150F4CFE881F9818C859D8548
:10400000AE85BF85892B8A2B8B2B41F480859185CA
:10401000A285B3858C879D87AE87BF87418169E480
:10402000CE010E946F0BCFB7F8948091B20481113A
:1040300027C0EBE0F3E08491EFE1F3E09491E82F07
:10404000F0E0EE0FFF1FED51FD4FA591B491EC9103
:10405000E92321F461E08AE00E948E0A61E08AE0AF
:104060000E94BC0A8CB580618CBD8CB580648CBD0F
:1040700061E08DE00E94BC0A61E08BE00E94BC0A16
:104080008091B2048F5F8093B204CFBF81E099CF5B
:10409000E881F981E485E15090E0E33020F4F0E03C
:1040A000E552FE4F90810C851D852E853F8540E0B1
:1040B00052E16AE770E080E004171507260737072A
:1040C00040F476956795579547958F5F8630A1F7B1
:1040D00087E09C709065282F2695922B80958170A3
:1040E0009CBD8DBDE881F981408169E4CE010E94CB
:1040F0006F0BA881B981EA85FB8530E020E012963C
:104100004C916CE2CE010995C1CFA881B981EA85B5
:10411000FB8530E020E013964C916CE20995E88134
:10412000F981418169E458CF0C940232FF920F93D8
:104130001F93CF93DF93EC01F62E08811981C801FC
:104140000E94F431F81621F06F2DC8010E9402324E
:10415000CE01DF91CF911F910F91FF900895EF92C3
:10416000FF920F931F93CF93DF9300D0CDB7DEB7AD
:1041700080E0E82E85E0F82E00E110E01A83098344
:10418000F70161917F01CE0101960E9496200F5F99
:104190001F4F0431110591F780E095E00F900F90CB
:1041A000DF91CF911F910F91FF90EF900895EF92C3
:1041B000FF920F931F93CF93DF9300D0CDB7DEB75D
:1041C0008CEFE82E84E0F82E06E210E01A830983D3
:1041D000F70161917F01CE0101960E9496200F5F49
:1041E0001F4F0A32110591F78CEF94E00F900F905A
:1041F000DF91CF911F910F91FF90EF900895EF9273
:10420000FF920F931F93CF93DF9300D0CDB7DEB70C
:1042100080EFE82E84E0F82E0CE210E01A83098388
:10422000F70161917F01CE0101960E9496200F5FF8
:104230001F4F0833110591F780EF94E00F900F9016
:10424000DF91CF911F910F91FF90EF900895AF9262
:10425000BF92CF92DF92EF92FF920F931F93CF9373
:10426000DF9300D0CDB7DEB78B016B0124E0C20E27
:10427000D11C7B015C01A61AB70AC5018E0D9F1DDA
:104280009A838983F70161917F01CE0101960E9493
:104290009620EC14FD0489F7C8010F900F90DF9170
:1042A000CF911F910F91FF90EF90DF90CF90BF9033
:1042B000AF900895CF93DF93C9E0D1E0688182E0A9
:1042C00090E00E949420698183E090E00E94942015
:1042D0006AEC74E088E190E00E9427216EEC74E0C3
:1042E0008CE190E00E94272165E071E084E090E09D
:1042F0000E94272162EE74E08CE390E00E94272167
:104300006EED74E080E490E00E9427216AED74E095
:1043100084E490E00E9427210E94AF206091D204A3
:1043200085E290E00E9494200E94D72061E48AE216
:1043300090E00E94942062E48BE290E00E9494203E
:10434000DF91CF910C94FF201092EC0480E09DE26D
:10435000A1E3B1E08093CA049093CB04A093CC0472
:10436000B093CD0480E49BE4ACE4B0E08093CE0451
:104370009093CF04A093D004B093D104E0EFF4E085
:1043800080E494E5A9E8B0E080839183A283B383BD
:104390008CE599EFAAE4B0E084839583A683B78384
:1043A00084E195E0ABE4B0E080879187A287B38792
:1043B00080E696E5ACE6B0E08093E2049093E304F7
:1043C000A093E404B093E50440E25DE16AE970E0A3
:1043D0004093DE045093DF046093E0047093E104A3
:1043E00040EC5CEA68ED70E04093DA045093DB0443
:1043F0006093DC047093DD048093050190930601C3
:10440000A0930701B093080180E090E0A0E7B1E439
:104410008093FC049093FD04A093FE04B093FF04EA
:1044200081E08093D20446E950E060E070E0409380
:104430000005509301056093020570930305809376
:10444000C6040E945A216091C60490E080E00C945A
:104450009420DF92EF92FF920F931F93CF93DF93FD
:10446000CDB7DEB72A970FB6F894DEBF0FBECDBF2B
:10447000FC018B0180E289838A838B838C838EE2AB
:10448000D82EDE8283818F9382818F9381818F9357
:1044900080818F9389E892E09F938F931F936F930E
:1044A0000E94F636F80101900020E9F7CF0101974C
:1044B000801B910B0FB6F894DEBF0FBECDBF8630C8
:1044C00009F457C0C4F4853009F442C01A86BE010D
:1044D0006F5F7F4FC8010E94E0362A960FB6F894AE
:1044E000DEBF0FBECDBFDF91CF911F910F91FF9027
:1044F000EF90DF900895873009F448C0883031F795
:1045000042E050E0B801CE0101960E94E7368CE20D
:104510008B837801F2E0EF0EF11C43E050E0B7012D
:10452000CE0104960E94E736DF8242E050E0B801F7
:104530006B5F7F4FCE0108960E94E7368091EF04B3
:10454000863021F646E050E0B701CE0104960EC059
:1045500042E050E0B801CE0104960E94E73643E005
:1045600050E0B8016E5F7F4FCE0107960E94E7369C
:10457000ADCF43E050E0B801CE0103960E94E7368C
:1045800043E050E0B8016D5F7F4FEECFF8018191BD
:10459000BF0189838CE28A8343E050E0CE01039619
:1045A0000E94E73643E050E0B8016C5F7F4FDCCFFC
:1045B000BF92CF92DF92EF92FF920F931F93CF9310
:1045C000DF93CDB7DEB760970FB6F894DEBF0FBEAE
:1045D000CDBFE091EF04EA3008F034C1F0E0ED50D7
:1045E000FD4D0C940134FD22FD223D24502457241E
:1045F00022246524BE24F8243B258091EC048823E2
:1046000009F4BEC0813009F4C3C0609167047091A1
:1046100068048091690490916A048E01055F1F4FC0
:1046200021E042E00E949F2F86E58F87188A81E073
:1046300096E00E94111F2CE0F22E36E0E32E0E943D
:10464000261E82E691E00E947B0FAE014F5F5F4F16
:1046500068E180E00E94A8148DE393E00E947B0F44
:10466000E091E904EE2309F499C0F0E0E75FFE4F22
:10467000808190E00396F89EA001F99E500D1124D0
:1046800045595E4F68E282E00E94A8148091D304ED
:10469000882351F08091C804882331F049EA53E01F
:1046A00068E288E40E94A8148091ED04813051F4FE
:1046B0008091C804882331F044EA53E068E288E43A
:1046C0000E94A8148091ED04813051F48091D304AC
:1046D000882331F049EA53E068E288E40E94A81494
:1046E0008091ED04833051F48091C804882331F027
:1046F00049EA53E068E288E40E94A8148091C80463
:10470000811106C04DE852E068E288E40E94A814D6
:104710008091C604882309F447C08091C404E1E174
:10472000F1E010E09191891718F01F5F1C30D1F76C
:104730001E9DA0011124435E5E4F68E281E60E9447
:10474000A8140BE02EE64AE266E081E096E00E94C3
:10475000991098E0C92EB12CB11671F18CE2D82EC7
:1047600000E027E04D2D6C2D81E096E00E94370E91
:10477000D39423E3D212F4CFB39489E0C80EECCFE4
:10478000BE016F5F7F4F85E091E00E9429223DCFFF
:10479000BE016F5F7F4F86ED94E0F7CF4091090136
:1047A0004F9DA00111246CCF00E020E842E360E0BF
:1047B00081E096E00E94370E8091EE0440E952E0DD
:1047C00081111DC08091E6044FE952E08823B9F0C1
:1047D0004091D6045091D7046091D8047091D904C7
:1047E0008091050190910601A0910701B091080107
:1047F000481759076A077B07A9F543E952E060E4C7
:1048000082E00E94A8148091E60442EA52E08111FD
:1048100002C04AEA52E060E480E20E94A81480915B
:10482000C604882339F0AE01455F5F4F60E48AE536
:104830000E94A8140E94261E81E096E00E94E71EB6
:104840008111FDCE60960FB6F894DEBF0FBECDBFCE
:10485000DF91CF911F910F91FF90EF90DF90CF905C
:10486000BF90089584179507A607B70718F447E97E
:1048700052E0C5CF4BE952E0C2CF8DE393E00E94F6
:104880007B0F6091E8048091E90442EB52E08111D2
:1048900002C042EF52E08DEE92E00E94231FD2CF81
:1048A0004FE253E06091E8048AE693E0F6CF60912E
:1048B000E8048091D40443E753E0833019F48DE792
:1048C00093E0EBCF89E893E0E8CF8091C90424E03E
:1048D000829FC0011124BE016F5F7F4F80519B4FAB
:1048E0000E94292281E096E00E94111F1CE045E908
:1048F00053E06EE08AE00E94A8148091C9048130E0
:10490000B9F178F18230B9F100E020E842E160E0ED
:1049100081E096E00E94370E82E691E00E947B0FD4
:10492000AE014F5F5F4F6EE280E00E94A8148DE3FE
:1049300093E00E947B0FE091E904F0E0E75FFE4F17
:104940004081419FA001112445595E4F6CE385E0F1
:104950000E94A81481E096E00E94E71E8111C7CF53
:1049600071CF4EE953E06EE08AE50E94A814CCCFE7
:1049700043EA53E0F8CF48EA53E0F5CF609167048B
:10498000709168048091690490916A048E01055FBA
:104990001F4F21E042E00E949F2F86E58F87188AF3
:1049A00081E096E00E94111F4DEA53E06EE08AE03C
:1049B0000E94A81400E020E842E160E081E096E077
:1049C0000E94370E82E691E00E947B0FAE01455FA8
:1049D0005F4F6EE284E10E94A8148DE393E00E9491
:1049E0007B0F81E096E00E94E71E8111DDCF2ACF88
:1049F000809103058F93809102058F93809101052B
:104A00008F93809100058F938BEB93E09F938F930F
:104A10007E018BE0E80EF11CFF92EF920E94F636C9
:104A200081E096E00E94111F0FB6F894DEBF0FBE22
:104A3000CDBF4EEB53E06EE085E00E94A81400E08D
:104A400020E842E160E081E096E00E94370E82E6D5
:104A500091E00E947B0FA7016EE284E10E94A814FE
:104A60008DE393E00E947B0F81E096E00E94E71EB9
:104A70008111DFCFE7CE4DEC53E06091E80487EE83
:104A800093E00BCFCF93DF93E091D504AFEFAE0F60
:104A9000B0E0AE5ABB4FAC91A093E904B0E0A75F81
:104AA000BE4FCEEFCE0FD0E0CE5ADB4F88818C9335
:104AB000ADEFAE0FB0E0AE5ABB4F8C918093EF04D8
:104AC000ACEFAE0FB0E0AE5ABB4F8C918093E804D0
:104AD000E550E093D504F0E0EE5AFB4F80818093DF
:104AE000E704DF91CF910C94D8229091EB04191632
:104AF00094F491E09093EB049091EB042091E804FE
:104B0000920F9093E8041092EB04891730F480938D
:104B1000E8040C94D8229FEFEDCF9111FACF81E0F9
:104B2000F6CF1F920F920FB60F9211242F933F933F
:104B30008F939F93AF93BF938091B4049091B504EA
:104B4000A091B604B091B7043091B30423E0230FD1
:104B50002D3758F50196A11DB11D2093B304809304
:104B6000B4049093B504A093B604B093B7048091B5
:104B7000B8049091B904A091BA04B091BB04019615
:104B8000A11DB11D8093B8049093B904A093BA04F9
:104B9000B093BB04BF91AF919F918F913F912F91A3
:104BA0000F900FBE0F901F90189526E8230F0296C6
:104BB000A11DB11DD2CF1F920F920FB60F921124DB
:104BC0002F933F934F935F936F937F938F939F9315
:104BD000AF93BF93EF93FF938091B900887F8036A6
:104BE00009F44AC0F0F5883209F4A7C018F58031FD
:104BF00009F49BC0B8F4882309F4F9C0883009F49B
:104C000094C0FF91EF91BF91AF919F918F917F9150
:104C10006F915F914F913F912F910F900FBE0F9029
:104C20001F901895883109F488C0803251F780931D
:104C30004A0514C0803409F49DC040F48033B9F3B0
:104C40008833F9F680934A0585ECB0C0803509F4C5
:104C500085C0883509F496C0883499F60E943311CE
:104C6000D0CF883909F48CC038F5883729F050F452
:104C7000883611F0803729F683E080934C05109236
:104C8000B10457C0883809F47BC0803919F08038E6
:104C900009F0B7CF8091B104803208F071C0E09183
:104CA000B10481E08E0F8093B1048091BB00F0E0ED
:104CB000EF56FB4F80833DC0803B39F0E0F4803AF3
:104CC00009F479C0883A09F09CCF84E080934C05C0
:104CD00010928E0410928D04E0918B04F0918C045C
:104CE000099580918D0481110FC081E080938D041E
:104CF00010926B0409C0803C09F4A6CF883C09F4EB
:104D0000A3CF883B09F07DCFE0918E0481E08E0F28
:104D100080938E04F0E0E559FB4F80818093BB00C7
:104D200090918E0480918D0429C0809127058093F5
:104D3000BB0085EC8093BC0064CF909149058091C5
:104D40004805981758F5E091490581E08E0F80934A
:104D50004905F0E0E85DFA4F8081E9CFE09149052F
:104D600081E08E0F809349058091BB00F0E0E85D03
:104D7000FA4F808390914905809148059817C8F2B1
:104D800085E8D8CFE091490581E08E0F80934905F1
:104D90008091BB00F0E0E85DFA4F808380914B0585
:104DA00081115CCF81E08093260584EA8093BC006A
:104DB00010924C0526CF85EC8093BC0010924C05D8
:104DC0008091B104803230F4E091B104F0E0EF560C
:104DD000FB4F10826091B10470E0E0918F04F0917C
:104DE000900481E994E009951092B1040ACF1092E1
:104DF0004A0534CF1F920F920FB60F9211242F93B2
:104E00003F934F935F936F937F938F939F93AF9352
:104E1000BF93CF93DF93EF93FF93F89480917B063A
:104E20000E94650AEC0180917A060E94650A9091C1
:104E300079069F70CC0FDD1FC82B24E0929FC00124
:104E4000112481549E4FC80FD92FD11D8881809382
:104E500079068073803129F5809162048F5F809399
:104E60006204109261049091E704891770F1109226
:104E700062048091EB048F5F8093EB04FF91EF91CC
:104E8000DF91CF91BF91AF919F918F917F916F9162
:104E90005F914F913F912F910F900FBE0F901F90F8
:104EA0001895803291F4809161048F5F8093610442
:104EB000109262049091E704891738F0109261040F
:104EC0008091EB0481508093EB047894D7CF1092BB
:104ED00074051092730588EE93E0A0E0B0E0809333
:104EE000750590937605A0937705B093780589E6CC
:104EF00092E0909372058093710588E08093B406E8
:104F00008093B5061092AD061092AE061092AF06D1
:104F100010928506109286061092870610928806D7
:104F20001092890610928A0610928B0610928C06B7
:104F300010928D0610928E0610928F061092900697
:104F40001092910610929206109293061092940677
:104F50001092950610929606109297061092980657
:104F60001092990610929A0610929B0610929C0637
:104F700010929D0610929E0610929F061092A00617
:104F80001092A1061092A2061092A3061092A406F7
:104F90001092A5061092A6061092A7061092A806D7
:104FA0001092A9061092AA061092AB061092AC06B7
:104FB00080E498E7ADE7B1E08093B6069093B7063A
:104FC000A093B806B093B90683E080937A0682E096
:104FD00080937B0660E083E00E94BC0A60E08091E1
:104FE0007B060E94BC0A61E080917A060E948E0ACC
:104FF00061E080917B060E948E0A109279061092E1
:1050000000061092FF0586E696E090937606809360
:105010007506109277061092780610921A068BE7A2
:1050200092E09093FE058093FD0510920206109287
:105030000106109216061092190610920D06109293
:105040000E0610920F06109210068FEF809317062F
:1050500080931C06E0E2F6E086E396E02FEF2193D2
:105060008E179F07E1F78DEE9BE0909306068093E5
:1050700005068CEB9CE0909308068093070682ED72
:105080009FE190930A068093090688EC90E1909343
:105090000C0680930B0630E020E040E069E081E000
:1050A00096E00E94ED0B10924A061092490680E1AC
:1050B0009EE090933706809336068DE795E09093B7
:1050C0003B0680933A0681E080933C0610923D06B1
:1050D000109256061092720680937306809374069F
:1050E00083E892E0909339068093380681E096E059
:1050F0000E94DA0DE0913806F09139060280F381C2
:10510000E02D81E096E0099582E796E090934C06C9
:1051100080934B0688E0809329068AE080932A06D4
:1051200089E080932B060895789484B5826084BDCD
:1051300084B5816084BD85B5826085BD85B581609B
:1051400085BD80916E00816080936E001092810019
:1051500080918100826080938100809181008160D4
:105160008093810080918000816080938000809195
:10517000B10084608093B1008091B0008160809321
:10518000B00080917A00846080937A0080917A00E8
:10519000826080937A0080917A00816080937A00A7
:1051A00080917A00806880937A001092C10062E05A
:1051B00082E00E94BC0A62E083E00E94BC0A62E0D6
:1051C00086E00E94BC0A62E084E00E94BC0A60E0C3
:1051D0008EE00E94BC0A60E08FE00E94BC0A61E0A1
:1051E00085E00E94BC0A61E081E10E94BC0A62E0A5
:1051F00087E00E94BC0A61E08CE00E94BC0A62E089
:1052000080E10E94BC0A61E08CE00E948E0A68EC9A
:1052100070E080E090E00E942F0B80916800846035
:105220008093680080916D008C6080936D0078940D
:1052300083E08093090181E080930A011092E904E0
:105240008AE290E00E94D01E813409F04EC18BE2C8
:1052500090E00E94D01E823409F047C190E080E0C7
:105260000E94D01E8093C60482E090E00E94D01E6F
:105270008093090183E090E00E94D01E80930A0190
:105280006AEC74E088E190E00E94AA1E6EEC74E083
:105290008CE190E00E94AA1E65E071E084E090E05D
:1052A0000E94AA1E62EE74E08CE390E00E94AA1EA7
:1052B0006EED74E080E490E00E94AA1E6AED74E056
:1052C00084E490E00E94AA1E85E290E00E94D01E35
:1052D0008093D2040E94591E0E94751E0E94911E46
:1052E000E0910506F091060630E020E040E06AE03B
:1052F00081E096E0099581E096E00E94111F81E02F
:1053000096E00E94E71E8111FACF60E081E096E00E
:105310000E942A10E0910506F091060630E020E098
:1053200040E06BE081E096E0099580910501909165
:105330000601A0910701B09108018093D6049093D3
:10534000D704A093D804B093D9041092EC0481E060
:105350008093E7041092EF041092D5048093E80440
:105360000E949F1D61E08CE00E948E0A84E00E94F2
:10537000650A892B31F50E941E0A81E096E00E94A1
:10538000111F8DE393E00E947B0F41EF53E068E132
:1053900084E10E94A81441E054E06CE284E10E94A0
:1053A000A81481E096E00E94E71E8111EACF0E94D6
:1053B000A4210E94181C68EB7BE080E090E00E9432
:1053C0002F0B84E00E94650A892B51F46091C6047A
:1053D00081E068276093C60490E080E00E949420FA
:1053E0000E941E0A81E096E00E94111F8DE393E067
:1053F0000E947B0F40E154E068E184E10E94A81420
:105400004EE154E06CE284E10E94A81481E096E051
:105410000E94E71E8111EACF60ED77E080E090E026
:105420000E942F0B80E10E94650A21E0892B09F47C
:1054300020E02093C8040E94D82250E5C52E53ECEA
:10544000D52EE12CF12C11E060E5862E63EC962E32
:10545000A12CB12C04E035E0232E47E0342E0E942D
:105460000A0B4090BC045090BD046090BE04709044
:10547000BF049B01AC0124193509460957092901CC
:105480003A0130E1431637E253066104710408F42F
:10549000C5C06093BC047093BD048093BE04909318
:1054A000BF048091C204843029F1853009F439C0E9
:1054B00081113DC084E00E94650A892B11F410938C
:1054C000C204E091EF04EA3008F055C0F0E0E5597D
:1054D000F54D0C9401349D2A662C822C752DC02D1F
:1054E0003A2E512EF62E2D2F8A2F0E94A4210E9493
:1054F0005A21F6CE84E00E94650A892B69F48091D6
:10550000C0048F5F8093C0048832D8F282E0809319
:10551000C1042092C204D5CF1093C1041092C204DA
:10552000D0CF84E00E94650A892B59F2F7CF8F5FB4
:105530008093C2041092C004C4CF86E00E94650A22
:1055400021E0009709F020E02093EE04892B09F078
:105550006FC08091ED04833031F463E070E081E04E
:1055600090E00E9425131092EC040E94181C0E94E7
:10557000D8221093EF0480E10E94650A21E0892B74
:1055800009F420E02093C8048091C704281751F043
:105590001092D3040E94D8220E94181C8091C80443
:1055A0008093C7040E94261E8091C6048823D9F0E8
:1055B0008091C5048F5F8093C50460E50E94BF336E
:1055C000911111C08FE00E94F80A959587959595E5
:1055D00087958093C4040E9425128091EF04811165
:1055E00002C00E94D8228091C304811106C060E0ED
:1055F0008CE00E948E0A1093C3048091C504833608
:1056000068F01092C5048091EA04882339F0815033
:105610008093EA04811102C00E945A210E94261E32
:1056200020E030E0232B09F41ACF0E94000012CFB3
:1056300070E060E081E090E00E9425138091EB042F
:105640008823C1F1E091E904E13009F046C0E0911E
:105650000A0144E0E49FF0011124E15BFD4F8081E9
:105660009181A281B3818093010190930201A09363
:105670000301B0930401A091EB042091010130914A
:10568000020140910301509104010A2E000CBB0B52
:105690000E9412342091EC04222351F1213009F4AC
:1056A00095C01092EB040E94181C83E08093EA04DA
:1056B0000E94D8220E944712C82F813009F4F4C0FA
:1056C000823009F058CF0E944D121093E804C09325
:1056D000EF0483E08093E704F4C0F0E0E75FFE4F5F
:1056E000E08154E0E59FF0011124ED5BFD4FB7CF61
:1056F0002091EB0440900501509006016090070155
:105700007090080127FF55C09B01AC0197FF07C0AF
:1057100022273327A901261B370B480B590B2415C9
:1057200035054605570508F444C08092050190925E
:105730000601A0920701B09208018091CA049091DD
:10574000CB04A091CC04B091CD04409105015091BF
:105750000601609107017091080184179507A6075B
:10576000B70740F48093050190930601A0930701C9
:10577000B09308018091CE049091CF04A091D00401
:10578000B091D1044091050150910601609107014B
:1057900070910801481759076A077B0708F081CF05
:1057A0008093050190930601A0930701B09308012F
:1057B00078CF460E571E681E791E40920501509202
:1057C00006016092070170920801B7CF2091EB04A7
:1057D0004090D6045090D7046090D8047090D904BB
:1057E00027FF11C09B01AC0197FF07C02227332779
:1057F000A901261B370B480B590B24153505460507
:10580000570508F048C0460E571E681E791E409284
:10581000D6045092D7046092D8047092D904809133
:10582000CA049091CB04A091CC04B091CD044091D6
:10583000D6045091D7046091D8047091D90484178C
:105840009507A607B70740F48093D6049093D70432
:10585000A093D804B093D9048091CE049091CF0442
:10586000A091D004B091D1044091D6045091D704B6
:105870006091D8047091D904481759076A077B07CB
:1058800008F00FCF8093D6049093D704A093D80448
:10589000B093D90406CF8092D6049092D704A092F8
:1058A000D804B092D904BBCFE091E904F0E0E75FFF
:1058B000FE4F80818F5F843038F4808383E0809353
:1058C000EA040E94D82257CEC083F8CF86E00E9417
:1058D000650A21E0009709F020E02093EE04892B6F
:1058E00009F449CE8091E604882349F01093EC0432
:1058F0000E94181C0E94D8221092EF043CCE1092F5
:10590000EC04F6CF8091EB04882319F086E00E9426
:1059100075250E944712C82F813009F02CCE809146
:10592000E804833009F4AEC030F5813079F182307B
:1059300009F021CE8091ED04813009F07CC0809186
:10594000050190910601A0910701B0910801809393
:10595000E2049093E304A093E404B093E50483E0AD
:105960008093ED048091DA049091DB04A091DC0433
:10597000B091DD0429C0853009F4AFC008F4A1C09E
:10598000863009F0F8CD0E944225F5CD8091ED04D6
:10599000813059F58091050190910601A091070190
:1059A000B09108018093E2049093E304A093E4048F
:1059B000B093E5041093ED048091E2049091E30428
:1059C000A091E404B091E504809305019093060151
:1059D000A0930701B09308011092E6041092EC0422
:1059E0000E94181C0E945A21CECF823089F48091E7
:1059F000050190910601A0910701B09108018093E3
:105A0000DE049093DF04A093E004B093E104D2CFCE
:105A1000833081F68091050190910601A0910701E4
:105A2000B09108018093DA049093DB04A093DC0426
:105A3000B093DD04BFCF823089F48091050190914D
:105A40000601A0910701B09108018093DE049093B4
:105A5000DF04A093E004B093E10481CF833009F028
:105A60007ECF8091050190910601A0910701B09130
:105A700008018093DA049093DB04A093DC04B093D4
:105A8000DD046DCF8091E6048C278093E6048823A3
:105A9000A9F0C093EC048091050190910601A091BA
:105AA0000701B09108018093D6049093D704A09386
:105AB000D804B093D9040E94181C65CF1092EC044E
:105AC000FACF1092D5048091E9048C278093E904E1
:105AD0001092EF04C093E704F4CE0E944D1283E0CD
:105AE0008093EF04C093E804ECCE8091EB0488230C
:105AF00019F085E00E9475250E944712882309F459
:105B00003ACDC091E804C33051F1C0F4C130E1F0A6
:105B1000C23009F030CD0E944D1289E08093EF042D
:105B2000E091E904F0E0E75FFE4FC0831093E804E2
:105B30000E94D82283E08093E7041DCDC430C9F0D1
:105B4000C53009F420CF17CD0E944D120093EF0409
:105B500082E08093E80483E08093D404B2CE0E9474
:105B60004D1298E09093EF040E94D8221093E7041E
:105B700002CD0E944D121093E7043092EF04A1CEA3
:105B80008091EB04882319F082E00E9475250E9421
:105B90004712882309F4EFCCC091E804C130A9F082
:105BA000C23009F0E8CCE091D404E150E73008F0CD
:105BB000EACEF0E0E252F24D0C9401340D2E1A2E92
:105BC000272E2A2E2D2E302E332E8091D404853070
:105BD000F1F040F4833091F0843009F0D4CE0E948B
:105BE000FF2069CF8630B1F0873009F0CCCE6091CC
:105BF000D20485E290E00E9494205DCF80E10E9473
:105C0000650A019709F057CFC093D30454CF0E947F
:105C1000D720B9CE0E94AF20B6CE8CE190E00E9492
:105C2000FC316093CE047093CF048093D0049093A2
:105C3000D104A9CE88E190E00E94FC316093CA04AF
:105C40007093CB048093CC049093CD049CCE10929F
:105C5000D30431CF0E94911E2ECF0E94751E93CE89
:105C60000E94591E90CE85E290E00E94D01E809343
:105C7000D20421CF8091EB04882319F084E00E94A4
:105C800075250E944712882309F475CC8091E80499
:105C90008093D2040093EF041093E8043092D4046C
:105CA00010CE8091EB04882309F455C0E091C9041B
:105CB000A091E904B0E0A75FBE4FAC9124E0A29FA1
:105CC000D0011124AD5BBD4F2D913D914D915C9163
:105CD000209301013093020140930301509304018A
:105CE000A091EB048091EB0494E0E99FF001112472
:105CF000EF01C051DB4F488059806A807B8087FF6D
:105D00003BC00A2E000CBB0B0E9412349B01AC015D
:105D100097FF07C022273327A901261B370B480B03
:105D2000590BE051FB4F241535054605570528F062
:105D3000C082D182E282F38208C0460E571E681EDE
:105D4000791E40825182628273821092EB040E941B
:105D5000181C0E94D8220E9447128130D1F1823053
:105D600009F009CC83E08093E7040093EF041093DB
:105D7000E8040093D404A5CDA091EB040A2E000CF6
:105D8000BB0B0E941234460E571E681E791EA1EFEF
:105D90004A16A9EB5A06A5EF6A06A5E07A0680F432
:105DA000488259826A827B82E051FB4F80819181D7
:105DB000A281B3818035934CA105B10530F6B8CFEF
:105DC00020E63AE544EF55E0288339834A835B8334
:105DD000EBCFE091E904F0E0E75FFE4F80818F5F59
:105DE000873010F480836DCD10826BCD0E94251218
:105DF0000E94D8228091EB048823E1F02091EB04EB
:105E00006091FC047091FD048091FE049091FF0468
:105E10001216E4F42DEC3CEC4CEC5DE30E9458329D
:105E20006093FC047093FD048093FE049093FF0440
:105E30001092EB040E944712882309F49CCB009334
:105E4000EF041093E8042092D4043BCD2DEC3CECFD
:105E50004CEC5DE30E945732E3CF8091EB04882342
:105E600009F44BC04091EB04042E000C550B660B5B
:105E7000770B8091000590910105A0910205B091EA
:105E80000305841B950BA60BB70B8093000590931D
:105E90000105A0930205B09303051092EB04813D28
:105EA0009740A105B10564F080ED97E0A0E0B0E077
:105EB0008093000590930105A0930205B09303051C
:105EC0008091000590910105A0910205B091030514
:105ED0008033984FAF4FBF4F64F480E398EFAFEF3C
:105EE000BFEF8093000590930105A0930205B09346
:105EF00003050E949F1D0E94D8220E9447128823FA
:105F000009F439CB0093EF041093E80496E09093E2
:105F1000D404D7CC8091EB04882319F083E00E944D
:105F200075250E944712882309F425CB8091E80447
:105F300081508093C904A6E0A093EF04C2CCEF92F5
:105F40000F931F93CF93DF93E80134E047FD34E1D3
:105F5000042E000C550B57FF03C051954195510974
:105F6000E32E022F242FAE010E94BD2FCE01DF9120
:105F7000CF911F910F91EF900895A9E0B0E0E3EC6D
:105F8000FFE20C9426326A01F22EB02E102FFBE3B2
:105F9000AF2EA01608F41BE31F5F012F27E0AE0110
:105FA0004F5F5F4F0E941C31BC018981982F99700F
:105FB000913009F43FC09BE2E1FC04C09E2D91703A
:105FC000E0FC3AC05E2D5071E82FE87083FF46C0B8
:105FD00084E0911101C083E0EF2DE81B8F1508F0DC
:105FE000E0E0D6018E2F20E2552351F1992329F0CC
:105FF000D6019C93C60101966C0196012D5F3F4F1F
:10600000E2FE24C08EE4D6018C9391E411969C9319
:10601000119712968C93D9018E2F90E281111BC09B
:10602000E20FF32FF11D10828EEF9FEF2996ECE027
:106030000C9442329DE2C6CF90E2C4CF2D938150A2
:106040008111FCCFCE0ED11CE0E0D0CF8EE6D60180
:106050008C9391E6DBCF9D938150E0CF482F447025
:1060600082FF3DC084E0911101C083E08F1510F4E0
:10607000EF2DE81BD6018E2F20E2552309F199233D
:1060800029F0D6019C93C60101966C0196012D5F03
:106090003F4FE2FE1BC089E4D6018C938EE411963B
:1060A0008C93119786E412968C93D9018E2F90E2EF
:1060B000882309F4B5CF9D938150FACF2D93815059
:1060C0008111FCCFCE0ED11CE0E0D9CF89E6D601FC
:1060D0008C938EE611968C93119786E6E4CF9B0104
:1060E00077FF02C030E020E0A1E0B0E0911102C0F3
:1060F000B0E0A0E0F9013196AE0FBF1F8B2C912CC0
:10610000BB2009F461C05401EFEFAE1ABE0AAA0D1C
:10611000BB1DFA161B0619F014F04F2D4A1B511126
:1061200088C0E3FC59C07601A42FB0E2A1114FC092
:10613000C40ED11C992309F45BC040E0D60111962E
:10614000F60190836D01552309F448C0012F060F15
:106150009A81582F507184FF03C0913309F4015084
:1061600010160CF047C0093008F008E0EEE2FE2EF1
:106170005B01A01AB10885019194819491082F3F89
:10618000320729F4D601FC92F60131966F016217AD
:10619000730794F1021713077CF5DB01A21BB30B05
:1061A000AA24A394B12CAC0EBD1EAA0DBB1D119642
:1061B0008C9121503109D601119628153905F4F03A
:1061C000F60180836D01DBCFB12CA12CA0CFF701AC
:1061D000B1937F01A150AACF9111B0CFD601942FD6
:1061E00050E302C05D9391509111FCCFC40ED11CBD
:1061F00040E0ACCF01E0BACF80E3DBCF621773079A
:1062000031F4963388F4953311F4552369F0F6018F
:106210008083FD01842F90E2811108C0A40FB11D7D
:106220001C9290E080E002CF81E3F1CF9193815006
:10623000F3CF911183CF8ACF283008F027E033279E
:10624000DA01990F311D87FD916000966105710596
:1062500039F432602E5F3D9330E32A95E1F70895DB
:106260009F3F30F080387105610509F03C5F3C5F6D
:106270003D93913008F08068911DDF93CF931F9379
:106280000F93FF92EF92192F987F9695E92F96958D
:106290009695E90FFF27EE53FF4F99273327EE24FA
:1062A000FF24A701E70105900894079428F4360F0E
:1062B000E71EF81E491F511D660F771F881F991F83
:1062C0000694A1F70590079428F4E70EF81E491FDD
:1062D000561FC11D770F881F991F661F0694A1F7CF
:1062E0000590079428F4F80E491F561FC71FD11DAB
:1062F000880F991F661F771F0694A1F705900794D2
:1063000020F4490F561FC71FD81F990F661F771F0C
:10631000881F0694A9F784911095177041F0D695BF
:10632000C79557954795F794E7941A95C1F7E8E60E
:10633000F0E06894159015913591659195910590CF
:106340007FE27395E118F10A430B560BC90BD00994
:10635000C0F7E10CF11E431F561FC91FD01D7EF46C
:10636000703311F48A95E6CFE894015030F0080FAD
:106370000AF40027021708F4202F2395022F7A33FE
:1063800028F079E37D932A95E9F710C07D932A954B
:1063900089F6069497956795379517951794E118A0
:1063A000F10A430B560BC90BD00998F023957E9147
:1063B00073957A3308F070E37C932013B8F77E91DD
:1063C00070617D9330F0839571E37D9370E32A953E
:1063D000E1F71124EF90FF900F911F91CF91DF9182
:1063E000992787FD90950895F999FECF92BD81BDBB
:1063F000F89A992780B50895A6E1B0E044E050E00E
:106400000C941232262FF999FECF1FBA92BD81BD8E
:1064100020BD0FB6F894FA9AF99A0FBE0196089526
:10642000DC01CB01FC01F999FECF06C0F2BDE1BD54
:10643000F89A319600B40D9241505040B8F7089543
:106440002F923F924F925F926F927F928F929F9284
:10645000AF92BF92CF92DF92EF92FF920F931F9372
:10646000CF93DF93CDB7DEB7CA1BDB0B0FB6F89423
:10647000DEBF0FBECDBF09942A88398848885F8463
:106480006E847D848C849B84AA84B984C884DF80D4
:10649000EE80FD800C811B81AA81B981CE0FD11DB8
:1064A0000FB6F894DEBF0FBECDBFED010895505872
:1064B000BB27AA270E946F320C9418330E940A331C
:1064C00038F00E94113320F039F49F3F19F426F47C
:1064D0000C9407330EF4E095E7FB0C940133E92F9D
:1064E0000E94293358F3BA17620773078407950788
:1064F00020F079F4A6F50C944B330EF4E0950B2EB6
:10650000BA2FA02D0B01B90190010C01CA01A00105
:106510001124FF27591B99F0593F50F4503E68F160
:106520001A16F040A22F232F342F4427585FF3CFA1
:10653000469537952795A795F0405395C9F77EF472
:106540001F16BA0B620B730B840BBAF09150A1F0BB
:10655000FF0FBB1F661F771F881FC2F70EC0BA0F41
:10656000621F731F841F48F4879577956795B795C9
:10657000F7959E3F08F0B0CF9395880F08F09927C4
:10658000EE0F979587950895E89409C097FB3EF420
:1065900090958095709561957F4F8F4F9F4F992370
:1065A000A9F0F92F96E9BB279395F69587957795EE
:1065B0006795B795F111F8CFFAF4BB0F11F460FFAE
:1065C0001BC06F5F7F4F8F4F9F4F16C0882311F006
:1065D00096E911C0772321F09EE8872F762F05C01A
:1065E000662371F096E8862F70E060E02AF09A95B5
:1065F000660F771F881FDAF7880F9695879597F9AA
:10660000089597F99F6780E870E060E008959FEF34
:1066100080EC089500240A94161617061806090639
:10662000089500240A941216130614060506089508
:10663000092E0394000C11F4882352F0BB0F40F490
:10664000BF2B11F460FF04C06F5F7F4F8F4F9F4FD0
:10665000089557FD9058440F551F59F05F3F71F052
:106660004795880F97FB991F61F09F3F79F08795B9
:106670000895121613061406551FF2CF4695F1DF42
:1066800008C0161617061806991FF1CF86957105D2
:10669000610508940895E894BB2766277727CB0106
:1066A00097F908950E9465330C9418330E940A33B9
:1066B00038F00E94113320F0952311F00C9401332F
:1066C0000C94073311240C944C330E94293370F33B
:1066D000959FC1F3950F50E0551F629FF001729F87
:1066E000BB27F00DB11D639FAA27F00DB11DAA1F96
:1066F000649F6627B00DA11D661F829F2227B00DE3
:10670000A11D621F739FB00DA11D621F839FA00D6D
:10671000611D221F749F3327A00D611D231F849FBD
:10672000600D211D822F762F6A2F11249F57504014
:106730009AF0F1F088234AF0EE0FFF1FBB1F661F8F
:10674000771F881F91505040A9F79E3F510580F058
:106750000C9401330C944C335F3FE4F3983ED4F334
:10676000869577956795B795F795E7959F5FC1F7FC
:10677000FE2B880F911D9695879597F90895991B83
:1067800079E004C0991F961708F0961B881F7A9528
:10679000C9F78095089597FB072E16F4009407D04B
:1067A00077FD09D00E94913507FC05D03EF4909505
:1067B00081959F4F0895709561957F4F0895A1E24F
:1067C0001A2EAA1BBB1BFD010DC0AA1FBB1FEE1F6B
:1067D000FF1FA217B307E407F50720F0A21BB30BB6
:1067E000E40BF50B661F771F881F991F1A9469F732
:1067F00060957095809590959B01AC01BD01CF018E
:106800000895EE0FFF1F0590F491E02D09940E946A
:10681000A535A59F900DB49F900DA49F800D911D4F
:1068200011240895B7FF0C9407340E940734821B8B
:10683000930B0895DF93CF931F930F939A9DF02DA1
:10684000219FF00D8B9DF00D8A9DE02DF10D039F92
:10685000F00D029FE00DF11D4E9DE00DF11D5E9DBE
:10686000F00D4F9DF00D7F936F93BF92AF925F93AA
:106870004F93D5010E94A5358B01AC01D7010E9431
:10688000A535EB01E80FF91FD6010E9469342F915D
:106890003F91D6010E94A535C60FD71FE81FF91FEB
:1068A000AF91BF910E9469342F913F910E94A5350D
:1068B000C60FD71FE81FF91FD6010E94A535E60FA6
:1068C000F71F9801BE01CF010F911F91CF91DF916A
:1068D00008950E94A535460F571FC81FD91F08F4F9
:1068E00031960895E894DF93CF93FC01DB010E9479
:1068F000A5357F936F93E9019A01AC01BF93AF93E4
:106900003F932F93DF010E94A53526F46C1B7D0B6E
:10691000820B930B9E01EB01FC010E946934AF9145
:10692000BF912F913F910E946934BE01CF01F901BF
:106930002F913F91CF91DF910895689401C0E89421
:10694000F92FF12B12F00C94D134A0E0B0E0EBEA77
:10695000F4E30C942632092E059422F40E942D357E
:10696000112392F4F0E80F26FFEFE094F0940095E5
:106970001095B094C094D094A194BF0ACF0ADF0AB6
:10698000EF0AFF0A0F0B1F0B0E94DC3407FC0E946A
:106990002D35CDB7DEB7ECE00C944232689401C0DF
:1069A000E8948F929F92CF93DF930E94DC34DF9123
:1069B000CF919F908F90089588249924F401E40149
:1069C000B0E49F93AA279A158B049C04ED05FE055D
:1069D000CF05D007A10798F4AD2FDC2FCF2FFE2FC6
:1069E000E92D982C892E982F872F762F652F542FDD
:1069F000432F322F2227B85031F7BF9127C01B2ECB
:106A0000BF91BB27220F331F441F551F661F771FDF
:106A1000881F991F881C991CEE1FFF1FCC1FDD1FAC
:106A2000AA1FBB1F8A149B04EC05FD05CE05DF05DC
:106A3000A007B10748F08A189B08EC09FD09CE09A8
:106A4000DF09A00BB10B21601A94E1F62EF494013A
:106A5000AF01BE01CD01000C089560957095809541
:106A6000909530954095509521953F4F4F4F5F4FF2
:106A70006F4F7F4F8F4F9F4F0895002E083090F03B
:106A8000982F872F762F652F542F432F322F2227B1
:106A90000850F4CF220F331F441F551F661F771F66
:106AA000881F991F0A95B2F7002D089597FD10943D
:106AB000002E083098F00850232F342F452F562FE2
:106AC000672F782F892F912DF4CF1594979587955F
:106AD0007795679557954795379527950A95AAF71E
:106AE0001124002D08952A0D3B1D4C1D5D1D6E1DAA
:106AF0007F1D801F911F08952A153B054C055D05DC
:106B00006E057F058007910708950024A7FD009476
:106B10002A17300540055005600570058005900571
:106B20000895AA1BBB1B51E107C0AA1FBB1FA617D4
:106B3000B70710F0A61BB70B881F991F5A95A9F726
:106B400080959095BC01CD010895A29FB001B39F9F
:106B5000C001A39F700D811D1124911DB29F700D66
:106B6000811D1124911D08950F931F93CF93DF93DF
:106B70008230910510F482E090E0E091BC06F09143
:106B8000BD0630E020E0B0E0A0E0309799F4211598
:106B9000310509F44AC0281B390B24303105D8F5DA
:106BA0008A819B816115710589F1FB019383828341
:106BB000FE0111C04081518102811381481759079C
:106BC000E0F04817590799F4109761F012960C936A
:106BD000129713961C933296CF01DF91CF911F919C
:106BE0000F9108950093BC061093BD06F4CF2115B4
:106BF000310551F04217530738F0A901DB019A0122
:106C0000BD01DF01F801C1CFEF01F9CF9093BD06BF
:106C10008093BC06CDCFFE01E20FF31F81939193C9
:106C20002250310939832883D7CF2091BA06309179
:106C3000BB06232B41F420910D0130910E013093BE
:106C4000BB062093BA0620910B0130910C0121154F
:106C5000310541F42DB73EB740910F01509110011D
:106C6000241B350BE091BA06F091BB06E217F3073F
:106C7000A0F42E1B3F0B2817390778F0AC014E5FAC
:106C80005F4F2417350748F04E0F5F1F5093BB0628
:106C90004093BA06819391939FCFF0E0E0E09CCFC0
:106CA000CF93DF930097E9F0FC01329713821282B1
:106CB000A091BC06B091BD06ED0130E020E0109738
:106CC000A1F420813181820F931F2091BA06309167
:106CD000BB062817390709F061C0F093BB06E093A3
:106CE000BA06DF91CF910895EA01CE17DF07E8F5E4
:106CF0004A815B819E0141155105B1F7E901FB8392
:106D0000EA8349915991C40FD51FEC17FD0761F42F
:106D1000808191810296840F951FE9019983888370
:106D2000828193819B838A83F0E0E0E012968D91CB
:106D30009C9113970097B9F52D913C911197CD0136
:106D40000296820F931F2091BA063091BB06281736
:106D5000390739F6309751F51092BD061092BC06EE
:106D6000B093BB06A093BA06BCCFD383C283408145
:106D70005181840F951FC817D90761F44E5F5F4F8B
:106D800088819981480F591F518340838A819B8153
:106D9000938382832115310509F0B0CFF093BD06AE
:106DA000E093BC069ECFFD01DC01C0CF13821282AE
:106DB000D7CFDC0101C06D9341505040E0F70895FA
:106DC000FB01DC0101900D920020E1F70895FB0129
:106DD000DC014150504048F001900D920020C9F76D
:106DE00001C01D9241505040E0F70895AEE0B0E080
:106DF000ECEFF6E30C942E320D891E8986E08C832D
:106E00001A8309838FEF9FE79E838D83AE01475ED0
:106E10005F4F6F89788DCE0101960E9419372F81BF
:106E20003885020F131FF80110822E96E4E00C94AF
:106E30004A32ABE0B0E0EFE1F7E30C9420327C01A2
:106E40003B018A01FC0117821682838181FFC8C140
:106E5000CE0101965C01F7019381F30193FD8591C9
:106E600093FF81913F01882309F453C1853239F49E
:106E700093FD859193FF81913F01853229F4B701FC
:106E800090E00E940939E7CF912C212C312CFFE1B1
:106E9000F31538F08B3211F190F4803209F183321E
:106EA00029F137FC3CC020ED280F2A3050F536FE82
:106EB00020C08AE0989E200D1124922E06C08D32AB
:106EC00091F0803371F7689430F8F30193FD859168
:106ED00093FF81913F018111DACF21C0689431F88D
:106EE000689432F8F2CF689433F8EFCF689434F8AE
:106EF000ECCFEAE02E9E200D1124222E689435F866
:106F0000E4CF8E3229F436FC04C1689436F8DDCF24
:106F10008C3619F4689437F8D8CF8836B1F2982FA8
:106F20009F7D95549330E0F08336A1F18337C1F112
:106F3000833509F063C02801F2E04F0E511CF801BF
:106F4000C080D180692D70E036FC02C06FEF7FEF0A
:106F5000C6010E94F3384C01689437F882010AC0D8
:106F60000C5F1F4FFFE3F98388248394912C650104
:106F7000E89437F833FE2DC0522C8114910471F53A
:106F8000552009F468CFB70180E290E00E940939EA
:106F90005A94F6CFF801808189830E5F1F4FE4CFAA
:106FA0002801F2E04F0E511CF801C080D180692DFC
:106FB00070E036FC02C06FEF7FEFC6010E94FE3822
:106FC0004C018201D5CFB70180E290E00E940939DF
:106FD0002A942814190409F0B0F7CECFF60137FC33
:106FE000859137FE81916F01B70190E00E940939C8
:106FF00051105A94F1E08F1A9108BFCF843619F0DE
:10700000893609F077C0F80137FE6BC06081718165
:10701000828193810C5F1F4FF32DFF763F2E97FFE8
:1070200009C090958095709561957F4F8F4F9F4FC8
:10703000689437F82AE030E0A5010E943939C82E5B
:10704000CA188C2C432C36FE0CC0E89440F8C914A6
:1070500040F434FE05C032FC03C0F32DFE7E4F2EFB
:10706000892C44FE95C0FE01EC0DF11D808180331A
:1070700009F087C0242D297E422E842D8870582E39
:1070800043FC95C040FE8FC09C2C821418F42C0C3D
:10709000922C981844FE91C0B70180E390E00E94C2
:1070A000093942FE09C088E790E041FE02C088E548
:1070B00090E0B7010E940939C91408F48AC0CA9443
:1070C000D12C9FEFC91AD90ACA0CDB1CF601829198
:1070D0006F01B70190E00E940939AC14BD04B1F70B
:1070E0004FCF60817181072E000C880B990B0E5FCA
:1070F0001F4F92CFD32CE894D4F82AE030E08537A4
:1071000039F1232D297FD22E8F3601F148F48835AD
:10711000A9F0F701868197812B96E2E10C943C322D
:10712000803749F08837A9F7D4FE02C06894D2F8B6
:1071300020E130E00DC06894D4F8F6CF34FE03C0EF
:10714000822F8660D82E20E132E002C028E030E0B5
:10715000F801D7FE0FC060817181828193810C5F3D
:107160001F4FA5010E943939C82ECA183D2CE8943A
:1071700037F867CF6081718190E080E00E5F1F4F2C
:10718000F0CF42FC02C0839478CF8394839475CF70
:10719000842D867809F471CFF6CFB70180E290E0B4
:1071A0000E94093983948214C0F3512C73CF522C5E
:1071B0005818821408F46ECFF8CF842D867809F41D
:1071C0007BCF8BE241FE80E247FC8DE2B70190E08D
:1071D00071CFB70180E390E00E9409399A946CCF97
:1071E0008FEF9FEF99CFFC01059061507040011027
:1071F000D8F7809590958E0F9F1F0895FC016150E0
:10720000704001900110D8F7809590958E0F9F1FC8
:1072100008950F931F93CF93DF93182F092FEB013E
:107220008B8181FD09C01FEF0FEF812F902FDF9120
:10723000CF911F910F91089582FF14C02E813F813D
:107240008C819D81281739073CF4E881F981CF01B1
:1072500001969983888310838E819F8101969F83F5
:107260008E83E3CFE885F985812F0995892BA1F3DA
:10727000DACFFA01AA27283051F1203181F1E894C0
:107280006F936E7F6E5F7F4F8F4F9F4FAF4FB1E019
:107290003ED0B4E03CD0670F781F891F9A1FA11D14
:1072A000680F791F8A1F911DA11D6A0F711D811D15
:1072B000911DA11D20D009F468943F912AE0269FDA
:1072C00011243019305D3193DEF6CF010895462F39
:1072D0004770405D4193B3E00FD0C9F7F6CF462F1A
:1072E0004F70405D4A3318F0495D31FD4052419383
:1072F00002D0A9F7EACFB4E0A69597958795779540
:107300006795BA95C9F700976105710508959B01C6
:10731000AC010A2E06945795479537952795BA954F
:10732000C9F7620F731F841F951FA01D0895F8945D
:02733000FFCF8D
:107332000564000000C0ACD80003010000BE068056
:107342000003050A0F14191E2832465A6920532DCC
:1073520030200020532D31200020532D32200020D8
:10736200532D33200020532D34200020532D35205F
:107372000020532D36200020532D37200020532D7E
:1073820038200020532D392000392B32302000398B
:107392002B34302000392B363020005354455020F6
:1073A20031487A2020200053544550203130487A09
:1073B2002020005354455020313030487A20005369
:1073C20054455020316B487A2020005354455020B8
:1073D20031306B487A200053544550203130306BA5
:1073E200487A005354455020314D487A20200000FD
:1073F2000204000300011003020000030201000660
:10740200000400060500200605040004080C1815F7
:10741200A015C019FF1815A115C819FF1815AE1926
:10742200FF1815AF19FF1815AE15D5168015A81639
:107432003F15D316001540158D161415201600158C
:10744200A115C815DA1612158116CF15D916F11520
:10745200DB1640152E15A415A619FF0001140A64A7
:1074620064323200093D00030428961008020280AB
:10747200004000010000000A00000064000000E873
:1074820003000010270000A086010040420F00DC2C
:107492000D620D350D00000000B6118911A61266AD
:1074A20011D106761167110000000012147D12A698
:1074B20012A512DA0D810D560D256C64004357009A
:1074C20054580052583D0052582B0052582D005229
:1074D2005800524954204F4E2000524954204F46E2
:1074E200460034304D2042414E440A32304D204253
:1074F200414E440A524954204F4E2F4F46460A31BC
:107502006B487A20313030487A203130487A0A5339
:10751200455454494E47530A45584954004D454E27
:10752200550034304D2042414E440A32304D204203
:10753200414E440A524954204F4E2F4F46460A317B
:107542004D487A203130306B487A2031306B487A9E
:107552000A53455454494E47530A45584954004426
:10756200494749204D4F44450A4946204652455114
:1075720055454E43590A43414C49425241544520D4
:107582005854414C0A43414C4942524154452056B9
:107592004F4C54530A455849540053455454494E8C
:1075A2004753004F4B0A43414E43454C0020444948
:1075B2004749204D4F44452000534156452F4341F2
:1075C2004E43454C002D2D2D46492D2D2D004D416C
:1075D200494E00204C534200205553420020562071
:1075E200434F5252454354494F4E00256400434194
:1075F2004C494252415445205854414C004D414956
:107602004E2049460A4C534220465245510A555390
:107612004220465245510053454C45435420494669
:1076220000524553455420504552464F524D454411
:107632000072656C6561736520627574746F6E00AB
:10764200204442343032302056322E3220007777B6
:0E765200772E6561336763792E636F6D0000DC
:00000001FF
